:020000040000FA
:1000000002EF00F00F013F0E926E000E936E000E95
:10001000946E030E956E0F0E966E000E386F000EE6
:10002000396F000E3A6F000E3B6F000E3C6F806A16
:10003000816A826A836A846A896A8A6A8B6A8C6A3C
:100040008D6A00018B8C006A016A026A036A046A85
:10005000056A066A076A086A096A0A6A0B6A0C6A0C
:100060000D6A0E6A0F6A106A116A126A136A146ABC
:10007000156A166A176A186A196A1A6A1B6A1C6A6C
:100080001D6A1E6A1F6A206A216A226A236A256A1B
:10009000266A276A296A246A286A2A6A2B6A2C6ACD
:1000A0002D6A2E6A2F6A306A316A326A336A346A7C
:1000B000356A366A376A386A396A3A6A3C6A3B6A2C
:1000C0003D6A3E6A3F6A406A416A426A436A446ADC
:1000D000456A466A476A486A496A4A6A4B6A4C6A8C
:1000E0004D6A4E6A506A516A526AD3EC35F0D3ECCD
:1000F00035F0D3EC35F0D3EC35F020EC2AF0C00E1F
:100100008A6E8C9C8C9E8C8A8C9A1FEC2BF03F0EF6
:100110008A6E8C9C8C9E8C8A8C9A42EC2BF08B8AFB
:1001200023EC2AF0FBEC35F0000EAA6E000EA96E4F
:10013000A69EA69CA68000000000A850116E000E8E
:10014000AA6E010EA96EA69EA69CA68000000000C5
:10015000A850126E000EAA6E020EA96EA69EA69C54
:10016000A68000000000A850136E000EAA6E030EB9
:10017000A96EA69EA69CA68000000000A850146E42
:10018000000EAA6E040EA96EA69EA69CA680000074
:100190000000A850156E000EAA6E050EA96EA69E50
:1001A000A69CA68000000000A850166E000EAA6E45
:1001B000060EA96EA69EA69CA68000000000A85070
:1001C000176E000EAA6E070EA96EA69EA69CA680AC
:1001D00000000000A850186E000EAA6E080EA96E4E
:1001E000A69EA69CA68000000000A850196E000ED6
:1001F000AA6E090EA96EA69EA69CA680000000000D
:10020000A8501A6E000EAA6E0A0EA96EA69EA69C93
:10021000A68000000000A8504C6E5FEC2BF0A4EC10
:100220002CF01D504E6E4CA41BEF01F083A21BEF6F
:1002300001F0AEEC34F0A4EC2CF080B280B63FEFCD
:1002400001F03EB640EF01F01550380B406E380E0D
:10025000405CD8B430EF01F0080E402632EF01F0D8
:10026000000E406E1550C70B156E405015124CB263
:10027000CBEC34F05FEC2BF03E8640EF01F03E9685
:1002800080B461EF01F03EB462EF01F01550380B1D
:10029000406E000E405CD8B452EF01F0080E405E94
:1002A00054EF01F0380E406E1550C70B156E4050DC
:1002B00015124CB2CBEC34F05FEC2BF03E8462EFC5
:1002C00001F03E944CB4A9EC34F080B279EF01F027
:1002D0003EB27AEF01F0040E415CD8B473EF01F046
:1002E000412A74EF01F0416A42EC2BF03E827AEF32
:1002F00001F03E92000E415CD8B495EF01F0010E82
:10030000415CD8B48AEF0BF0020E415CD8B4ACEF7C
:1003100011F0030E415CD8B48AEF20F0040E415C6A
:10032000D8B405EF26F01BEF01F01AEC2AF0410ECD
:1003300026EC2AF0B80E3FEC2AF0700E58EC2AF0AA
:10034000100E58EC2AF0100E58EC2AF0100E58EC53
:100350002AF0000E58EC2AF0F2EC44F0000E58ECB3
:100360002AF032EC44F0000E58EC2AF012EC44F083
:10037000000E58EC2AF032EC44F0000E58EC2AF053
:1003800072EC44F0000E58EC2AF032EC45F0000E0E
:1003900058EC2AF032EC44F0000E58EC2AF0F2EC63
:1003A00044F022EC47F002EC45F01DEC2AF0400E40
:1003B00026EC2AF0B80E3FEC2AF012EC45F0000EC5
:1003C00058EC2AF0F2EC43F0000E58EC2AF012EC54
:1003D00045F0000E58EC2AF022EC45F0000E58ECE7
:1003E0002AF002EC45F0000E58EC2AF0082A210E03
:1003F000085CD8B401EF02F0100E58EC2AF0F6EFCA
:1004000001F0086A700E58EC2AF01AEC2AF0400E3F
:1004100026EC2AF0BA0E3FEC2AF01DA82CEF02F0D1
:1004200022EC47F022EC47F022EC47F022EC47F0B8
:10043000000E58EC2AF022EC47F0000E58EC2AF09F
:1004400022EC47F0000E58EC2AF022EC47F0000EA8
:1004500058EC2AF056EF02F01BA478EF02F0FF0EE2
:1004600058EC2AF052EC46F0FF0E58EC2AF062EC01
:1004700046F0FF0E58EC2AF0FF0E58EC2AF0FF0E63
:1004800058EC2AF0A2EC46F0FF0E58EC2AF0A2EC51
:1004900045F0FF0E58EC2AF042EC46F0FF0E58EC07
:1004A0002AF0A2EC46F0FF0E58EC2AF0082A1A0EA9
:1004B000085CD8B461EF02F0000E58EC2AF056EF59
:1004C00002F0086A1DEC2AF0400E26EC2AF0BA0E63
:1004D0003FEC2AF0082A070E085CD8B475EF02F04A
:1004E000000E58EC2AF06AEF02F0086AFFEF02F003
:1004F000FF0E58EC2AF0A2EC46F0FF0E58EC2AF062
:10050000A2EC45F0FF0E58EC2AF042EC46F0FF0E4C
:1005100058EC2AF0A2EC46F0FF0E58EC2AF0000E40
:1005200058EC2AF0000E58EC2AF01BA2C8EF02F09B
:10053000FF0E58EC2AF062EC46F0FF0E58EC2AF061
:1005400092EC46F0FF0E58EC2AF002EC46F0FF0E5B
:1005500058EC2AF0E2EC45F0FF0E58EC2AF052EC91
:1005600046F0FF0E58EC2AF082EC45F0FF0E58ECF6
:100570002AF01DEC2AF0400E26EC2AF0BA0E3FECD1
:100580002AF032EC46F0FF0E58EC2AF0FFEF02F0B2
:10059000FF0E58EC2AF0A2EC45F0FF0E58EC2AF0C2
:1005A00062EC46F0FF0E58EC2AF072EC46F0FF0EBB
:1005B00058EC2AF002EC47F0FF0E58EC2AF0082A1B
:1005C0000D0E085CD8B4EAEF02F0000E58EC2AF0E9
:1005D000DFEF02F0086A1DEC2AF0400E26EC2AF04C
:1005E000BA0E3FEC2AF0082A070E085CD8B4FEEFDA
:1005F00002F0000E58EC2AF0F3EF02F0086A1DEC4E
:100600002AF0480E26EC2AF0BA0E3FEC2AF01DB86C
:1006100021EF03F01BA621EF03F0FF0E58EC2AF0A8
:1006200072EC46F0FF0E58EC2AF092EC46F0FF0E0A
:1006300058EC2AF062EC46F0FF0E58EC2AF02DEF51
:1006400003F0082A140E085CD8B42CEF03F0000E57
:1006500058EC2AF021EF03F0086A1DEC2AF05D0E39
:1006600026EC2AF0BA0E3FEC2AF01DB854EF03F046
:100670001BB054EF03F0FF0E58EC2AF0C2EC45F02B
:10068000FF0E58EC2AF042EC46F0FF0E58EC2AF030
:1006900072EC46F0FF0E58EC2AF0F2EC45F0FF0E3B
:1006A00058EC2AF060EF03F0082A1A0E085CD8B460
:1006B0005FEF03F0000E58EC2AF054EF03F0086AE5
:1006C0001AEC2AF0400E26EC2AF0B90E3FEC2AF084
:1006D0001DB8DFEF04F01CB679EF03F01CB8A7EFEC
:1006E00003F01CBAD5EF03F01CBC05EF04F0DFEFFC
:1006F00004F0FF0E58EC2AF0B2EC45F0FF0E58EC77
:100700002AF0B2EC46F0FF0E58EC2AF0A2EC46F0CC
:10071000FF0E58EC2AF0FF0E58EC2AF0FF0EA2EC68
:1007200045F0FF0E58EC2AF0B2EC45F0FF0E58EC05
:100730002AF0082A110E085CD8B4A4EF03F0000ECA
:1007400058EC2AF099EF03F0086AEBEF04F0FF0E83
:1007500058EC2AF0B2EC45F0FF0E58EC2AF0B2EC5F
:1007600046F0FF0E58EC2AF0A2EC46F0FF0E58ECD3
:100770002AF0FF0E58EC2AF0FF0E32EC46F0FF0E86
:1007800058EC2AF0B2EC45F0FF0E58EC2AF0082A9B
:10079000110E085CD8B4D2EF03F0000E58EC2AF02A
:1007A000C7EF03F0086AEBEF04F0FF0E58EC2AF0F5
:1007B00002EC46F0FF0E58EC2AF0C2EC45F0FF0EBA
:1007C00058EC2AF0A2EC45F0FF0E58EC2AF012EC9F
:1007D00042F0FF0E58EC2AF0C2EC41F0FF0E58EC4C
:1007E0002AF042EC42F0FF0E58EC2AF0E2EC41F025
:1007F000FF0E58EC2AF022EC42F0FF0E58EC2AF0E3
:10080000000E58EC2AF0EBEF04F0FF0E58EC2AF043
:1008100072EC46F0FF0E58EC2AF0A2EC45F0FF0E09
:1008200058EC2AF042EC46F0FF0E58EC2AF0000E8D
:1008300058EC2AF02B50526E529E010E525CD8B4E6
:100840003FEF04F0490E525CD8B467EF04F0030E9A
:10085000525CD8B48FEF04F0430E525CD8B4B7EFBB
:1008600004F0082A1E0E085CD8B43CEF04F0000E19
:1008700058EC2AF031EF04F0086AEBEF04F0000EB8
:1008800058EC2AF0FF0E58EC2AF0A2EC45F0FF0ECF
:1008900058EC2AF0B2EC45F0FF0E58EC2AF022ECAE
:1008A00047F0000E58EC2AF022EC47F0000E58EC0E
:1008B0002AF0000E58EC2AF0000E58EC2AF0000E38
:1008C00058EC2AF0000E58EC2AF0EBEF04F0000E82
:1008D00058EC2AF0FF0E58EC2AF042EC46F0FF0EDE
:1008E00058EC2AF0B2EC45F0FF0E58EC2AF022EC5E
:1008F00047F0000E58EC2AF022EC47F0000E58ECBE
:100900002AF0000E58EC2AF0000E58EC2AF0000EE7
:1009100058EC2AF0000E58EC2AF0EBEF04F0000E31
:1009200058EC2AF0FF0E58EC2AF0B2EC45F0FF0E1E
:1009300058EC2AF082EC45F0FF0E58EC2AF0B2ECAD
:1009400046F0FF0E58EC2AF022EC47F0000E58EC6F
:100950002AF0000E58EC2AF0000E58EC2AF0000E97
:1009600058EC2AF0000E58EC2AF0EBEF04F0000EE1
:1009700058EC2AF0FF0E58EC2AF0B2EC45F0FF0ECE
:1009800058EC2AF0A2EC45F0FF0E58EC2AF0A2EC4D
:1009900045F0FF0E58EC2AF022EC47F0000E58EC20
:1009A0002AF0000E58EC2AF0000E58EC2AF0000E47
:1009B00058EC2AF0000E58EC2AF0EBEF04F0082A6D
:1009C000320E085CD8B4EAEF04F0000E58EC2AF0BE
:1009D000DFEF04F0086A1AEC2AF0730E26EC2AF016
:1009E000B90E3FEC2AF01DB829EF05F01CA229EF43
:1009F00005F0FF0E58EC2AF0A2EC46F0FF0E58EC82
:100A00002AF002EC46F0FF0E58EC2AF01DEC2AF01A
:100A1000400E26EC2AF0B90E3FEC2AF032EC46F0FC
:100A2000FF0E58EC2AF0C2EC45F0FF0E58EC2AF00D
:100A300052EC46F0FF0E58EC2AF0A2EC45F0FF0E07
:100A400058EC2AF0C2EC45F0FF0E58EC2AF049EFC2
:100A500005F0082A0E0E085CD8B434EF05F0000E3D
:100A600058EC2AF029EF05F0086A1DEC2AF0400E38
:100A700026EC2AF0B90E3FEC2AF0082A1F0E085C7B
:100A8000D8B448EF05F0000E58EC2AF03DEF05F021
:100A9000086A1DEC2AF0600E26EC2AF0B90E3FEC35
:100AA0002AF01DB879EF05F01CA079EF05F0FF0ED4
:100AB00058EC2AF0F2EC45F0FF0E58EC2AF002EC6C
:100AC00046F0FF0E58EC2AF0FF0E58EC2AF0FF0E0D
:100AD00058EC2AF0D2EC45F0FF0E58EC2AF0A2ECCC
:100AE00046F0FF0E58EC2AF0000E58EC2AF085EF85
:100AF00005F0082A1C0E085CD8B484EF05F0000E3F
:100B000058EC2AF079EF05F0086A1AEC2AF0400E4A
:100B100026EC2AF0BB0E3FEC2AF04CB095EF05F026
:100B20001D504E6E4F6AAAEF05F01D504E5CD8A4C2
:100B30003F9A000E4F5CD8A4A0EF05F01D504E6EFA
:100B40003FBAAAEF05F0000E4E5CD8B4AAEF05F04C
:100B5000E8EC38F0000E4E5CD8A4B3EF05F066EC7C
:100B600039F0FDEF05F0400E4E5CD8A4BCEF05F067
:100B700086EC39F0FDEF05F0200E4E5CD8A4C5EFF1
:100B800005F0A7EC39F0FDEF05F0100E4E5CD8A48F
:100B9000CEEF05F0C8EC39F0FDEF05F0080E4E5C25
:100BA000D8A4D7EF05F000EC3AF0FDEF05F0020E07
:100BB0004E5CD8A4E0EF05F04EEC3AF0FDEF05F006
:100BC000010E4E5CD8A4E9EF05F09CEC3AF0FDEF85
:100BD00005F0FF0E58EC2AF01CEC3BF04E5019ECDF
:100BE00038F0FF0E58EC2AF0FF0E58EC2AF07BECA0
:100BF00038F022EC47F022EC47F01AEC2AF0400ED5
:100C000026EC2AF0BD0E3FEC2AF0000E58EC2AF03C
:100C100042EC44F0000E58EC2AF002EC45F0000ED5
:100C200058EC2AF0280E58EC2AF0280E58EC2AF03E
:100C3000280E58EC2AF0280E58EC2AF0280E58EC12
:100C40002AF0000E58EC2AF01AEC2AF0530E26EC8B
:100C50002AF0BD0E3FEC2AF05E0E295CD8A450EFBE
:100C600006F0000E58EC2AF022EC47F0000E58EC8B
:100C70002AF022EC47F0000E58EC2AF0000E58EC57
:100C80002AF0000E58EC2AF042EC41F0000E58EC2D
:100C90002AF032EC41F0000E58EC2AF075EF08F023
:100CA0005D0E295CD8A474EF06F0000E58EC2AF013
:100CB00022EC47F0000E58EC2AF022EC47F0000E30
:100CC00058EC2AF0000E58EC2AF0000E58EC2AF0EE
:100CD00042EC41F0000E58EC2AF032EC41F0000EEC
:100CE00058EC2AF075EF08F0440E295CD8A498EF70
:100CF00006F0000E58EC2AF022EC47F0000E58ECFB
:100D00002AF052EC41F0000E58EC2AF052EC41F07F
:100D1000000E58EC2AF0400E58EC2AF0000E58EC69
:100D20002AF022EC41F0000E58EC2AF075EF08F0A2
:100D3000450E295CD8A4BCEF06F0000E58EC2AF052
:100D400022EC47F0000E58EC2AF052EC41F0000E75
:100D500058EC2AF052EC41F0000E58EC2AF0400E0C
:100D600058EC2AF0000E58EC2AF022EC41F0000E6C
:100D700058EC2AF075EF08F03E0E295CD8A4E0EF9D
:100D800006F0000E58EC2AF022EC47F0000E58EC6A
:100D90002AF022EC47F0000E58EC2AF0000E58EC36
:100DA0002AF0000E58EC2AF052EC41F0000E58ECFC
:100DB0002AF092EC41F0000E58EC2AF075EF08F0A2
:100DC0003F0E295CD8A404EF07F0000E58EC2AF07F
:100DD00022EC47F0000E58EC2AF022EC47F0000E0F
:100DE00058EC2AF0000E58EC2AF0000E58EC2AF0CD
:100DF00052EC41F0000E58EC2AF092EC41F0000E5B
:100E000058EC2AF075EF08F0220E295CD8A428EFE0
:100E100007F0000E58EC2AF022EC47F0FF0E58ECD9
:100E20002AF032EC42F0FF0E58EC2AF032EC42F09D
:100E3000FF0E58EC2AF0BF0E58EC2AF0FF0E58ECCB
:100E40002AF0D2EC41F0FF0E58EC2AF075EF08F0D2
:100E5000230E295CD8A44CEF07F0000E58EC2AF0C2
:100E600022EC47F0FF0E58EC2AF032EC42F0FF0E75
:100E700058EC2AF032EC42F0FF0E58EC2AF0BF0E8C
:100E800058EC2AF0FF0E58EC2AF0D2EC41F0FF0E9D
:100E900058EC2AF075EF08F01F0E295CD8A470EF0B
:100EA00007F0000E58EC2AF022EC47F0000E58EC48
:100EB0002AF022EC47F0000E58EC2AF0000E58EC15
:100EC0002AF0FF0E58EC2AF042EC42F0FF0E58ECEC
:100ED0002AF012EC42F0FF0E58EC2AF075EF08F001
:100EE000200E295CD8A494EF07F0000E58EC2AF0ED
:100EF00022EC47F0000E58EC2AF022EC47F0000EEE
:100F000058EC2AF0000E58EC2AF0FF0E58EC2AF0AC
:100F100042EC42F0FF0E58EC2AF012EC42F0FF0EC9
:100F200058EC2AF075EF08F0110E295CD8A4B8EF40
:100F300007F0FF0E58EC2AF0C2EC41F0FF0E58EC1F
:100F40002AF022EC42F0FF0E58EC2AF012EC42F0AC
:100F5000FF0E58EC2AF0BF0E58EC2AF0FF0E58ECAA
:100F60002AF0F2EC41F0FF0E58EC2AF075EF08F091
:100F7000120E295CD8A4DCEF07F0FF0E58EC2AF023
:100F8000C2EC41F0FF0E58EC2AF022EC42F0FF0ECA
:100F900058EC2AF012EC42F0FF0E58EC2AF0BF0E8B
:100FA00058EC2AF0FF0E58EC2AF0F2EC41F0FF0E5C
:100FB00058EC2AF075EF08F0100E295CD8A400EF69
:100FC00008F0000E58EC2AF022EC47F0000E58EC26
:100FD0002AF0000E58EC2AF0FF0E58EC2AF0C2EC72
:100FE00041F0FF0E58EC2AF042EC42F0FF0E58ECB4
:100FF0002AF0D2EC41F0FF0E58EC2AF075EF08F021
:101000000F0E295CD8A424EF08F0000E58EC2AF04B
:1010100022EC47F0000E58EC2AF0000E58EC2AF0B3
:10102000FF0E58EC2AF0C2EC41F0FF0E58EC2AF00B
:1010300042EC42F0FF0E58EC2AF0D2EC41F0FF0EE9
:1010400058EC2AF075EF08F0000E58EC2AF0100E5C
:1010500058EC2AF0100E58EC2AF0100E58EC2AF03A
:10106000100E58EC2AF0100E58EC2AF0000E58EC36
:101070002AF0100E58EC2AF0100E58EC2AF0100E40
:1010800058EC2AF0100E58EC2AF0100E58EC2AF00A
:10109000000E58EC2AF0100E58EC2AF0100E58EC06
:1010A0002AF0100E58EC2AF0100E58EC2AF0100E10
:1010B00058EC2AF0000E58EC2AF0400E58EC2AF0BA
:1010C000000E58EC2AF0100E58EC2AF0100E58ECD6
:1010D0002AF0100E58EC2AF0100E58EC2AF0100EE0
:1010E00058EC2AF0000E58EC2AF0000E58EC2AF0CA
:1010F00082EC44F0000E58EC2AF062EC44F0000E52
:1011000058EC2AF072EC45F0000E58EC2AF01AEC7C
:101110002AF0400E26EC2AF0BC0E3FEC2AF0000E1E
:1011200058EC2AF072EC44F0000E58EC2AF0B2ECC5
:1011300044F0000E58EC2AF0280E58EC2AF0280E45
:1011400058EC2AF0280E58EC2AF0280E58EC2AF019
:10115000280E58EC2AF0000E58EC2AF01AEC2AF06F
:10116000530E26EC2AF0BC0E3FEC2AF01550380B3B
:10117000406E000E405CD8A4E6EF08F0000E58EC7C
:101180002AF0F2EC44F0000E58EC2AF052EC45F054
:10119000000E58EC2AF0D2EC44F0000E58EC2AF085
:1011A00012EC41F0000E58EC2AF022EC47F0000E51
:1011B00058EC2AF022EC47F0000E58EC2AF022EC12
:1011C00047F0000E58EC2AF031EF0AF0080E405CB0
:1011D000D8A413EF09F0000E58EC2AF0F2EC44F01A
:1011E000000E58EC2AF052EC45F0000E58EC2AF0B4
:1011F000D2EC44F0000E58EC2AF022EC41F0000E44
:1012000058EC2AF022EC47F0000E58EC2AF022ECC1
:1012100047F0000E58EC2AF022EC47F0000E58EC94
:101220002AF031EF0AF0100E405CD8A440EF09F02C
:10123000000E58EC2AF0F2EC44F0000E58EC2AF0C4
:1012400052EC45F0000E58EC2AF0D2EC44F0000EBF
:1012500058EC2AF032EC41F0000E58EC2AF022EC67
:1012600047F0000E58EC2AF022EC47F0000E58EC44
:101270002AF022EC47F0000E58EC2AF031EF0AF089
:10128000180E405CD8A484EF09F0000E58EC2AF048
:1012900022EC45F0000E58EC2AF002EC45F0000E6E
:1012A00058EC2AF002EC44F0000E58EC2AF022EC44
:1012B00047F083A270EF09F0FF0E58EC2AF082ECA1
:1012C00045F0FF0E58EC2AF0A2EC45F0FF0E58EC6A
:1012D0002AF0B2EC46F0FF0E58EC2AF031EF0AF09B
:1012E000000E58EC2AF002EC45F0000E58EC2AF003
:1012F000D2EC44F0000E58EC2AF022EC44F0000E40
:1013000058EC2AF031EF0AF0200E405CD8A4B1EF7F
:1013100009F0000E58EC2AF0F2EC44F0000E58EC04
:101320002AF052EC45F0000E58EC2AF0D2EC44F0D2
:10133000000E58EC2AF052EC41F0000E58EC2AF066
:1013400022EC47F0000E58EC2AF022EC47F0000E99
:1013500058EC2AF022EC47F0000E58EC2AF031EF5E
:101360000AF0280E405CD8A4DEEF09F0000E58EC1D
:101370002AF0F2EC44F0000E58EC2AF052EC45F062
:10138000000E58EC2AF0D2EC44F0000E58EC2AF093
:1013900062EC41F0000E58EC2AF022EC47F0000E0F
:1013A00058EC2AF022EC47F0000E58EC2AF022EC20
:1013B00047F0000E58EC2AF031EF0AF0300E405C96
:1013C000D8A40BEF0AF0000E58EC2AF0F2EC44F02F
:1013D000000E58EC2AF052EC45F0000E58EC2AF0C2
:1013E000D2EC44F0000E58EC2AF072EC41F0000E02
:1013F00058EC2AF022EC47F0000E58EC2AF022ECD0
:1014000047F0000E58EC2AF022EC47F0000E58ECA2
:101410002AF031EF0AF0000E58EC2AF0F2EC44F01A
:10142000000E58EC2AF052EC45F0000E58EC2AF071
:10143000D2EC44F0000E58EC2AF082EC41F0000EA1
:1014400058EC2AF022EC47F0000E58EC2AF022EC7F
:1014500047F0000E58EC2AF022EC47F0000E58EC52
:101460002AF01DA850921DB84CEF0AF0020E1F5C26
:10147000D8B458EF0AF0030E1F5CD8B458EF0AF046
:10148000010E1F5CD8B458EF0AF0210E1F5CD8B4CF
:1014900058EF0AF052EF0AF050B252EF0AF05FEC48
:1014A0002BF05082206A216A226A236A266A276A00
:1014B000205037EC38F01AEC2AF0400E26EC2AF0D7
:1014C000BE0E3FEC2AF0080E58EC2AF0F80E58EC4D
:1014D0002AF0080E58EC2AF0E00E58EC2AF0200E04
:1014E00058EC2AF0000E58EC2AF0000E58EC2AF0C6
:1014F000059C53EC38F0215037EC38F01AEC2AF008
:101500005A0E26EC2AF0BE0E3FEC2AF0F80E58ECEC
:101510002AF0000E58EC2AF0E00E58EC2AF0200ECB
:1015200058EC2AF0E00E58EC2AF0000E58EC2AF0A5
:10153000000E58EC2AF0059C53EC38F0225037ECA2
:1015400038F01AEC2AF0400E26EC2AF0BF0E3FECE1
:101550002AF0059C53EC38F042EC47F0235037EC6E
:1015600038F01AEC2AF04E0E26EC2AF0BF0E3FECB3
:101570002AF0059C53EC38F0265037EC38F01AEC82
:101580002AF05C0E26EC2AF0BF0E3FEC2AF0059CF8
:1015900053EC38F042EC47F0275037EC38F01AECB7
:1015A0002AF06A0E26EC2AF0BF0E3FEC2AF0059CCA
:1015B00053EC38F01DEC2AF0460E26EC2AF0BC0E57
:1015C0003FEC2AF0700E58EC2AF0100E58EC2AF07E
:1015D000100E58EC2AF0100E58EC2AF0000E58ECC1
:1015E0002AF052EC44F0000E58EC2AF0D2EC44F011
:1015F000000E58EC2AF0C2EC44F0000E58EC2AF031
:10160000082A220E085CD8B40BEF0BF0100E58EC31
:101610002AF000EF0BF0086A700E58EC2AF01DEC6F
:101620002AF0460E26EC2AF0BD0E3FEC2AF0000E02
:1016300058EC2AF012EC41F0000E58EC2AF0280E7B
:1016400058EC2AF0280E58EC2AF0280E58EC2AF014
:10165000280E58EC2AF0280E58EC2AF0000E58EC10
:101660002AF013500F0B406EEAEC2DF01DEC2AF01F
:10167000460E26EC2AF0BE0E3FEC2AF0000E58EC87
:101680002AF022EC41F0000E58EC2AF0280E58EC1B
:101690002AF0280E58EC2AF0280E58EC2AF0280ED2
:1016A00058EC2AF0280E58EC2AF0000E58EC2AF0DC
:1016B0001450F00B406E4042404240424042EAEC3F
:1016C0002DF01DEC2AF0460E26EC2AF0BF0E3FEC62
:1016D0002AF0000E58EC2AF032EC41F0000E58ECE3
:1016E0002AF0280E58EC2AF0280E58EC2AF0280E82
:1016F00058EC2AF0280E58EC2AF0280E58EC2AF064
:10170000000E58EC2AF014500F0B406EEAEC2DF04E
:101710001BEF01F04F6A1AEC2AF0410E26EC2AF07A
:10172000B80E3FEC2AF0700E58EC2AF0100E58EC70
:101730002AF0100E58EC2AF0100E58EC2AF0000E89
:1017400058EC2AF012EC44F0000E58EC2AF002ECAF
:1017500045F0000E58EC2AF092EC41F0000E58ECE7
:101760002AF052EC41F0000E58EC2AF022EC41F045
:10177000000E58EC2AF072EC41F0000E58EC2AF002
:1017800022EC47F0F2EC44F0000E58EC2AF032EC78
:1017900044F0000E58EC2AF052EC44F01DEC2AF014
:1017A000400E26EC2AF0B80E3FEC2AF0000E58EC62
:1017B0002AF072EC44F0000E58EC2AF002EC45F0EE
:1017C000000E58EC2AF012EC45F0000E58EC2AF00E
:1017D00032EC44F0000E58EC2AF0F2EC44F0000E2B
:1017E00058EC2AF0082A200E085CD8B4FDEF0BF064
:1017F000100E58EC2AF0F2EF0BF0086A700E58EC5D
:101800002AF01AEC2AF0410E26EC2AF0B90E3FEC31
:101810002AF0FF0E58EC2AF082EC45F0FF0E58EC4F
:101820002AF0B2EC45F0FF0E58EC2AF0B2EC45F08D
:10183000FF0E58EC2AF092EC46F0FF0E58EC2AF01E
:10184000C2EC45F0FF0E58EC2AF0A2EC46F0FF0E79
:1018500058EC2AF0A2EC46F0FF0E58EC2AF01DECF2
:101860002AF0410E26EC2AF0B90E3FEC2AF0FF0ECA
:1018700058EC2AF0B2EC45F0FF0E58EC2AF082EC5E
:1018800045F0FF0E58EC2AF0B2EC46F0FF0E58EC93
:101890002AF082EC45F0FF0E58EC2AF080B062EF9F
:1018A0000CF03EB063EF0CF0060E425CD8B45CEF77
:1018B0000CF0422A5DEF0CF0426A42EC2BF03E80C5
:1018C00063EF0CF03E9084B678EF0CF03EBC79EFFD
:1018D0000CF0000E425CD8B471EF0CF0420673EFCE
:1018E0000CF0060E426E42EC2BF03E8C79EF0CF0C1
:1018F0003E9C1AEC2AF0410E26EC2AF0BA0E3FEC80
:101900002AF0000E425CD8B4A6EF0CF0010E425C47
:10191000D8B46CEF0DF0020E425CD8B432EF0EF08A
:10192000030E425CD8B4F8EF0EF0040E425CD8B45B
:10193000BEEF0FF0050E425CD8B484EF10F0060E37
:10194000425CD8B44AEF11F0A8EF11F012EC41F06C
:10195000000E58EC2AF012EC41F0000E58EC2AF080
:1019600062EC44F0000E58EC2AF01DEC2AF0410E17
:1019700026EC2AF0BA0E3FEC2AF0115091EC38F028
:101980001AEC2AF0410E26EC2AF0BB0E3FEC2AF0AE
:1019900012EC41F0000E58EC2AF022EC41F0000E5F
:1019A00058EC2AF062EC44F0000E58EC2AF01DECE2
:1019B0002AF0410E26EC2AF0BB0E3FEC2AF0125022
:1019C00091EC38F01AEC2AF0410E26EC2AF0BC0E0D
:1019D0003FEC2AF012EC41F0000E58EC2AF032EC09
:1019E00041F0000E58EC2AF062EC44F0000E58EC86
:1019F0002AF01DEC2AF0410E26EC2AF0BC0E3FEC3A
:101A00002AF0135091EC38F01AEC2AF0410E26EC33
:101A10002AF0BD0E3FEC2AF012EC41F0000E58EC1B
:101A20002AF042EC41F0000E58EC2AF062EC44F04F
:101A3000000E58EC2AF01DEC2AF0410E26EC2AF09C
:101A4000BD0E3FEC2AF0145091EC38F01AEC2AF05D
:101A5000410E26EC2AF0BE0E3FEC2AF012EC41F0CB
:101A6000000E58EC2AF052EC41F0000E58EC2AF02F
:101A700062EC44F0000E58EC2AF01DEC2AF0410E06
:101A800026EC2AF0BE0E3FEC2AF0155091EC38F00F
:101A90001AEC2AF0410E26EC2AF0BF0E3FEC2AF099
:101AA00012EC41F0000E58EC2AF062EC41F0000E0E
:101AB00058EC2AF062EC44F0000E58EC2AF01DECD1
:101AC0002AF0410E26EC2AF0BF0E3FEC2AF0165009
:101AD00091EC38F0A8EF11F012EC41F0000E58EC48
:101AE0002AF072EC41F0000E58EC2AF062EC44F05F
:101AF000000E58EC2AF01DEC2AF0410E26EC2AF0DC
:101B0000BA0E3FEC2AF0175091EC38F01AEC2AF09C
:101B1000410E26EC2AF0BB0E3FEC2AF012EC41F00D
:101B2000000E58EC2AF082EC41F0000E58EC2AF03E
:101B300062EC44F0000E58EC2AF01DEC2AF0410E45
:101B400026EC2AF0BB0E3FEC2AF0185091EC38F04E
:101B50001AEC2AF0410E26EC2AF0BC0E3FEC2AF0DB
:101B600012EC41F0000E58EC2AF092EC41F0000E1D
:101B700058EC2AF062EC44F0000E58EC2AF01DEC10
:101B80002AF0410E26EC2AF0BC0E3FEC2AF0195048
:101B900091EC38F01AEC2AF0410E26EC2AF0BD0E3A
:101BA0003FEC2AF012EC41F0000E58EC2AF0A2ECC7
:101BB00041F0000E58EC2AF062EC44F0000E58ECB4
:101BC0002AF01DEC2AF0410E26EC2AF0BD0E3FEC67
:101BD0002AF01A5091EC38F01AEC2AF0410E26EC5B
:101BE0002AF0BE0E3FEC2AF012EC41F0000E58EC49
:101BF0002AF0F2EC43F0000E58EC2AF062EC44F0CC
:101C0000000E58EC2AF01DEC2AF0410E26EC2AF0CA
:101C1000BE0E3FEC2AF01B5091EC38F01AEC2AF083
:101C2000410E26EC2AF0BF0E3FEC2AF012EC41F0F8
:101C3000000E58EC2AF002EC44F0000E58EC2AF0AA
:101C400062EC44F0000E58EC2AF01DEC2AF0410E34
:101C500026EC2AF0BF0E3FEC2AF01C5091EC38F035
:101C6000A8EF11F012EC41F0000E58EC2AF012EC43
:101C700044F0000E58EC2AF062EC44F0000E58ECF0
:101C80002AF01DEC2AF0410E26EC2AF0BA0E3FECA9
:101C90002AF01D5091EC38F01AEC2AF0410E26EC97
:101CA0002AF0BB0E3FEC2AF012EC41F0000E58EC8B
:101CB0002AF022EC44F0000E58EC2AF062EC44F0DA
:101CC000000E58EC2AF01DEC2AF0410E26EC2AF00A
:101CD000BB0E3FEC2AF01E5091EC38F01AEC2AF0C3
:101CE000410E26EC2AF0BC0E3FEC2AF012EC41F03B
:101CF000000E58EC2AF032EC44F0000E58EC2AF0BA
:101D000062EC44F0000E58EC2AF01DEC2AF0410E73
:101D100026EC2AF0BC0E3FEC2AF01F5091EC38F074
:101D20001AEC2AF0410E26EC2AF0BD0E3FEC2AF008
:101D300012EC41F0000E58EC2AF042EC44F0000E98
:101D400058EC2AF062EC44F0000E58EC2AF01DEC3E
:101D50002AF0410E26EC2AF0BD0E3FEC2AF020506E
:101D600091EC38F01AEC2AF0410E26EC2AF0BE0E67
:101D70003FEC2AF022EC41F0000E58EC2AF012EC75
:101D800041F0000E58EC2AF062EC44F0000E58ECE2
:101D90002AF01DEC2AF0410E26EC2AF0BE0E3FEC94
:101DA0002AF0215091EC38F01AEC2AF0410E26EC82
:101DB0002AF0BF0E3FEC2AF022EC41F0000E58EC66
:101DC0002AF022EC41F0000E58EC2AF062EC44F0CC
:101DD000000E58EC2AF01DEC2AF0410E26EC2AF0F9
:101DE000BF0E3FEC2AF0225091EC38F0A8EF11F032
:101DF00022EC41F0000E58EC2AF032EC41F0000EDB
:101E000058EC2AF062EC44F0000E58EC2AF01DEC7D
:101E10002AF0410E26EC2AF0BA0E3FEC2AF02350AD
:101E200091EC38F01AEC2AF0410E26EC2AF0BB0EA9
:101E30003FEC2AF022EC41F0000E58EC2AF042EC84
:101E400041F0000E58EC2AF062EC44F0000E58EC21
:101E50002AF01DEC2AF0410E26EC2AF0BB0E3FECD6
:101E60002AF0245091EC38F01AEC2AF0410E26ECBE
:101E70002AF0BC0E3FEC2AF022EC41F0000E58ECA8
:101E80002AF052EC41F0000E58EC2AF062EC44F0DB
:101E9000000E58EC2AF01DEC2AF0410E26EC2AF038
:101EA000BC0E3FEC2AF0255091EC38F01AEC2AF0E9
:101EB000410E26EC2AF0BD0E3FEC2AF022EC41F058
:101EC000000E58EC2AF062EC41F0000E58EC2AF0BB
:101ED00062EC44F0000E58EC2AF01DEC2AF0410EA2
:101EE00026EC2AF0BD0E3FEC2AF0265091EC38F09B
:101EF0001AEC2AF0410E26EC2AF0BE0E3FEC2AF036
:101F000022EC41F0000E58EC2AF072EC41F0000E89
:101F100058EC2AF062EC44F0000E58EC2AF01DEC6C
:101F20002AF0410E26EC2AF0BE0E3FEC2AF0275094
:101F300091EC38F01AEC2AF0410E26EC2AF0BF0E94
:101F40003FEC2AF022EC41F0000E58EC2AF082EC33
:101F500041F0000E58EC2AF062EC44F0000E58EC10
:101F60002AF01DEC2AF0410E26EC2AF0BF0E3FECC1
:101F70002AF0285091EC38F0A8EF11F022EC41F053
:101F8000000E58EC2AF092EC41F0000E58EC2AF0CA
:101F900062EC44F0000E58EC2AF01DEC2AF0410EE1
:101FA00026EC2AF0BA0E3FEC2AF0295091EC38F0DA
:101FB0001AEC2AF0410E26EC2AF0BB0E3FEC2AF078
:101FC00022EC41F0000E58EC2AF0A2EC41F0000E99
:101FD00058EC2AF062EC44F0000E58EC2AF01DECAC
:101FE0002AF0410E26EC2AF0BB0E3FEC2AF02A50D4
:101FF00091EC38F01AEC2AF0410E26EC2AF0BC0ED7
:102000003FEC2AF022EC41F0000E58EC2AF0F2EC02
:1020100043F0000E58EC2AF062EC44F0000E58EC4D
:102020002AF01DEC2AF0410E26EC2AF0BC0E3FEC03
:102030002AF02B5091EC38F01AEC2AF0410E26ECE5
:102040002AF0BD0E3FEC2AF022EC41F0000E58ECD5
:102050002AF002EC44F0000E58EC2AF062EC44F056
:10206000000E58EC2AF01DEC2AF0410E26EC2AF066
:10207000BD0E3FEC2AF02C5091EC38F01AEC2AF00F
:10208000410E26EC2AF0BE0E3FEC2AF022EC41F085
:10209000000E58EC2AF012EC44F0000E58EC2AF036
:1020A00062EC44F0000E58EC2AF01DEC2AF0410ED0
:1020B00026EC2AF0BE0E3FEC2AF02D5091EC38F0C1
:1020C0001AEC2AF0410E26EC2AF0BF0E3FEC2AF063
:1020D00022EC41F0000E58EC2AF022EC44F0000E05
:1020E00058EC2AF062EC44F0000E58EC2AF01DEC9B
:1020F0002AF0410E26EC2AF0BF0E3FEC2AF02E50BB
:1021000091EC38F0A8EF11F022EC41F0000E58EC01
:102110002AF032EC44F0000E58EC2AF062EC44F065
:10212000000E58EC2AF01DEC2AF0410E26EC2AF0A5
:10213000BA0E3FEC2AF02F5091EC38F01AEC2AF04E
:10214000410E26EC2AF0BB0E3FEC2AF022EC41F0C7
:10215000000E58EC2AF042EC44F0000E58EC2AF045
:1021600062EC44F0000E58EC2AF01DEC2AF0410E0F
:1021700026EC2AF0BB0E3FEC2AF0305091EC38F000
:102180001AEC2AF0410E26EC2AF0BC0E3FEC2AF0A5
:1021900032EC41F0000E58EC2AF012EC41F0000E47
:1021A00058EC2AF062EC44F0000E58EC2AF01DECDA
:1021B0002AF0410E26EC2AF0BC0E3FEC2AF03150FA
:1021C00091EC38F01AEC2AF0410E26EC2AF0BD0E04
:1021D0003FEC2AF032EC41F0000E58EC2AF022ECF1
:1021E00041F0000E58EC2AF062EC44F0000E58EC7E
:1021F0002AF01DEC2AF0410E26EC2AF0BD0E3FEC31
:102200002AF0325091EC38F01AEC2AF0410E26EC0C
:102210002AF0BE0E3FEC2AF032EC41F0000E58ECF2
:102220002AF032EC41F0000E58EC2AF062EC44F057
:10223000000E58EC2AF01DEC2AF0410E26EC2AF094
:10224000BE0E3FEC2AF0335091EC38F01AEC2AF035
:10225000410E26EC2AF0BF0E3FEC2AF032EC41F0A2
:10226000000E58EC2AF042EC41F0000E58EC2AF037
:1022700062EC44F0000E58EC2AF01DEC2AF0410EFE
:1022800026EC2AF0BF0E3FEC2AF0345091EC38F0E7
:10229000A8EF11F032EC41F0000E58EC2AF052ECAD
:1022A00041F0000E58EC2AF062EC44F0000E58ECBD
:1022B0002AF01DEC2AF0410E26EC2AF0BA0E3FEC73
:1022C0002AF0355091EC38F01AEC2AF0410E26EC49
:1022D0002AF0BB0E3FEC2AF032EC41F0000E58EC35
:1022E0002AF062EC41F0000E58EC2AF062EC44F067
:1022F000000E58EC2AF01DEC2AF0410E26EC2AF0D4
:10230000BB0E3FEC2AF0365091EC38F01AEC2AF074
:10231000410E26EC2AF0BC0E3FEC2AF032EC41F0E4
:10232000000E58EC2AF072EC41F0000E58EC2AF046
:1023300062EC44F0000E58EC2AF01DEC2AF0410E3D
:1023400026EC2AF0BC0E3FEC2AF0375091EC38F026
:10235000DBEC2DF01BEF01F01AEC2AF0410E26EC1D
:102360002AF0B80E3FEC2AF0700E58EC2AF0100E4E
:1023700058EC2AF0100E58EC2AF0100E58EC2AF007
:10238000000E58EC2AF012EC44F0000E58EC2AF043
:1023900002EC45F0000E58EC2AF092EC41F0000EF1
:1023A00058EC2AF052EC41F0000E58EC2AF022ECE6
:1023B00041F0000E58EC2AF072EC41F0000E58EC9F
:1023C0002AF022EC47F002EC45F0000E58EC2AF01F
:1023D00032EC44F0000E58EC2AF012EC45F01DEC03
:1023E0002AF0400E26EC2AF0B80E3FEC2AF0000E40
:1023F00058EC2AF012EC45F0000E58EC2AF072EC82
:1024000044F0000E58EC2AF0B2EC44F0000E58EC08
:102410002AF052EC44F0000E58EC2AF0082A260E5E
:10242000085CD8B419EF12F0100E58EC2AF00EEF39
:1024300012F0086A700E58EC2AF0000E435CD8B413
:1024400029EF12F0010E435CD8B44BEF15F01BEFEF
:1024500001F01AEC2AF0460E26EC2AF0B90E3FECF9
:102460002AF002EC45F0000E58EC2AF032EC44F071
:10247000000E58EC2AF092EC44F0000E58EC2AF0D2
:1024800032EC44F0000E58EC2AF012EC44F0000E4E
:1024900058EC2AF012EC45F0000E58EC2AF022EC31
:1024A00047F0F2EC43F0000E58EC2AF022EC44F036
:1024B000000E58EC2AF022EC44F01DEC2AF0400EFD
:1024C00026EC2AF0B90E3FEC2AF0000E58EC2AF068
:1024D000F2EC44F0000E58EC2AF032EC44F0000E1E
:1024E00058EC2AF002EC45F0000E58EC2AF002EC11
:1024F00045F0000E58EC2AF080B08EEF12F03EB09E
:102500008FEF12F00A0E465CD8B48AEF12F0462A1A
:102510008BEF12F0466A3E808FEF12F03E9084B649
:10252000A2EF12F03EBCA3EF12F0000E465CD8B44E
:102530009DEF12F046069FEF12F00A0E466E3E8C9B
:10254000A3EF12F03E9C3F941AEC2AF04A0E26ECC0
:102550002AF0BB0E3FEC2AF0000E465CD8B4C5EF63
:1025600012F0000E58EC2AF012EC41F0000E58EC7C
:102570002AF012EC41F0000E58EC2AF062EC44F024
:10258000000E58EC2AF0D7EF12F0FF0E58EC2AF0AC
:10259000B2EC41F0FF0E58EC2AF0B2EC41F0FF0E25
:1025A00058EC2AF0F2EC45F0FF0E58EC2AF01AEC49
:1025B0002AF0670E26EC2AF0BB0E3FEC2AF0010E43
:1025C000465CD8B4F8EF12F0000E58EC2AF012EC8A
:1025D00041F0000E58EC2AF022EC41F0000E58ECCD
:1025E0002AF062EC44F0000E58EC2AF00AEF13F0E7
:1025F000FF0E58EC2AF0B2EC41F0FF0E58EC2AF036
:10260000C2EC41F0FF0E58EC2AF0F2EC45F0FF0E60
:1026100058EC2AF01DEC2AF0440E26EC2AF0BB0EF2
:102620003FEC2AF0020E465CD8B42BEF13F0000EFC
:1026300058EC2AF012EC41F0000E58EC2AF032EC83
:1026400041F0000E58EC2AF062EC44F0000E58EC19
:102650002AF03DEF13F0FF0E58EC2AF0B2EC41F0F7
:10266000FF0E58EC2AF0D2EC41F0FF0E58EC2AF0A5
:10267000F2EC45F0FF0E58EC2AF01DEC2AF0610E4A
:1026800026EC2AF0BB0E3FEC2AF0030E465CD8B4D1
:102690005EEF13F0000E58EC2AF012EC41F0000E41
:1026A00058EC2AF042EC41F0000E58EC2AF062ECB3
:1026B00044F0000E58EC2AF070EF13F0FF0E58ECC7
:1026C0002AF0B2EC41F0FF0E58EC2AF0E2EC41F0B7
:1026D000FF0E58EC2AF0F2EC45F0FF0E58EC2AF011
:1026E0001AEC2AF04A0E26EC2AF0BC0E3FEC2AF037
:1026F000040E465CD8B491EF13F0000E58EC2AF0AB
:1027000012EC41F0000E58EC2AF052EC41F0000EB1
:1027100058EC2AF062EC44F0000E58EC2AF0A3EFDB
:1027200013F0FF0E58EC2AF0B2EC41F0FF0E58EC1B
:102730002AF0F2EC41F0FF0E58EC2AF0F2EC45F0F2
:10274000FF0E58EC2AF01AEC2AF0670E26EC2AF05D
:10275000BC0E3FEC2AF0050E465CD8B4C4EF13F073
:10276000000E58EC2AF012EC41F0000E58EC2AF062
:1027700062EC41F0000E58EC2AF062EC44F0000EDE
:1027800058EC2AF0D6EF13F0FF0E58EC2AF0B2EC1A
:1027900041F0FF0E58EC2AF002EC42F0FF0E58EC2C
:1027A0002AF0F2EC45F0FF0E58EC2AF01DEC2AF06E
:1027B000440E26EC2AF0BC0E3FEC2AF0060E465CD6
:1027C000D8B4F7EF13F0000E58EC2AF012EC41F0F9
:1027D000000E58EC2AF072EC41F0000E58EC2AF092
:1027E00062EC44F0000E58EC2AF009EF14F0FF0EF2
:1027F00058EC2AF0B2EC41F0FF0E58EC2AF012EC43
:1028000042F0FF0E58EC2AF0F2EC45F0FF0E58ECC7
:102810002AF01DEC2AF0610E26EC2AF0B40E3FECF3
:102820002AF0070E465CD8B42AEF14F0000E58ECDC
:102830002AF012EC41F0000E58EC2AF082EC41F044
:10284000000E58EC2AF062EC44F0000E58EC2AF02E
:102850003CEF14F0FF0E58EC2AF0B2EC41F0FF0E02
:1028600058EC2AF022EC42F0FF0E58EC2AF0F2EC81
:1028700045F0FF0E58EC2AF01AEC2AF04A0E26EC2E
:102880002AF0BD0E3FEC2AF0080E465CD8B45DEF8E
:1028900014F0000E58EC2AF012EC41F0000E58EC47
:1028A0002AF092EC41F0000E58EC2AF062EC44F071
:1028B000000E58EC2AF06FEF14F0FF0E58EC2AF0DF
:1028C000B2EC41F0FF0E58EC2AF032EC42F0FF0E71
:1028D00058EC2AF0F2EC45F0FF0E58EC2AF01AEC16
:1028E0002AF0670E26EC2AF0BD0E3FEC2AF0090E06
:1028F000465CD8B490EF14F0000E58EC2AF012ECBD
:1029000041F0000E58EC2AF0A2EC41F0000E58EC19
:102910002AF062EC44F0000E58EC2AF0A2EF14F01A
:10292000FF0E58EC2AF0B2EC41F0FF0E58EC2AF002
:1029300042EC42F0FF0E58EC2AF0F2EC45F0FF0EAC
:1029400058EC2AF01AEC2AF04A0E26EC2AF0BF0EB8
:102950003FEC2AF00A0E465CD8B4F5EF14F0000EF6
:1029600058EC2AF022EC44F0000E58EC2AF032EC3D
:1029700044F0000E58EC2AF042EC44F0000E58EC03
:102980002AF0F2EC43F0000E58EC2AF022EC45F06D
:10299000000E58EC2AF092EC44F0000E58EC2AF0AD
:1029A00012EC45F0000E58EC2AF022EC47F092ECC5
:1029B00044F0000E58EC2AF01DEC2AF0400E26ECF4
:1029C0002AF0BF0E3FEC2AF0C2EC44F0000E58ECA7
:1029D0002AF0F2EC43F0000E58EC2AF022EC44F01E
:1029E000000E58EC2AF039EF15F0FF0E58EC2AF0E3
:1029F000B2EC45F0FF0E58EC2AF0C2EC45F0FF0EA9
:102A000058EC2AF0D2EC45F0FF0E58EC2AF082EC9C
:102A100045F0FF0E58EC2AF0C2EC46F0FF0E58ECE1
:102A20002AF032EC46F0FF0E58EC2AF0B2EC46F0F9
:102A3000FF0E58EC2AF032EC47F032EC46F0FF0E75
:102A400058EC2AF01DEC2AF0400E26EC2AF0BF0EBE
:102A50003FEC2AF062EC46F0FF0E58EC2AF082ECD4
:102A600045F0FF0E58EC2AF0B2EC45F0FF0E58ECA2
:102A70002AF0DBEC2DF080B848EF15F03EB849EFB6
:102A800015F0010E436E42EC2BF03E8849EF15F035
:102A90003E981BEF01F01AEC2AF0460E26EC2AF0C5
:102AA000B90E3FEC2AF0000E465CD8B487EF15F063
:102AB000010E465CD8B474EF16F0020E465CD8B432
:102AC000CDEF17F0030E465CD8B4E1EF18F0040E1A
:102AD000465CD8B4C5EF19F0050E465CD8B4D4EF07
:102AE0001AF0060E465CD8B4FBEF1BF0070E465CEE
:102AF000D8B45FEF1DF0080E465CD8B417EF1EF097
:102B0000090E465CD8B4CFEF1EF087EF1FF05FECE4
:102B10003BF03FB28EEF15F0050E496E3FB4DDEF8E
:102B200015F080B0B6EF15F03EB0B7EF15F0010E1E
:102B3000495CD8A4A0EF15F0080E496EB3EF15F06C
:102B4000040E495CD8A4A9EF15F0010E496EB3EF4D
:102B500015F0080E495CD8A4B2EF15F0050E496EC9
:102B6000B3EF15F049063E80B7EF15F03E9084B6FE
:102B7000DCEF15F03EBCDDEF15F0080E495CD8A483
:102B8000C6EF15F0010E496ED9EF15F0010E495C44
:102B9000D8A4CFEF15F0040E496ED9EF15F0050E4D
:102BA000495CD8A4D8EF15F0080E496ED9EF15F09E
:102BB000492A3E8CDDEF15F03E9C1AEC2AF0460EB9
:102BC00026EC2AF0BC0E3FEC2AF0010E495CD8B48A
:102BD00017EF16F0040E495CD8B43AEF16F0080E61
:102BE000495CD8B45BEF16F0FF0E58EC2AF0B2EC5B
:102BF00046F0FF0E58EC2AF092EC46F0FF0E58EC2F
:102C00002AF0C2EC46F0FF0E58EC2AF052EC46F0E7
:102C1000FF0E58EC2AF0A2EC45F0FF0E58EC2AF01B
:102C200022EC47F0000E58EC2AF05BEF16F0FF0E96
:102C300058EC2AF0D2EC45F0FF0E58EC2AF0A2EC4A
:102C400046F0FF0E58EC2AF0E2EC46F0FF0E58EC8E
:102C50002AF0A2EC45F0FF0E58EC2AF032EC46F0D8
:102C6000FF0E58EC2AF022EC46F0FF0E58EC2AF04A
:102C70005BEF16F0FF0E58EC2AF072EC46F0FF0EF8
:102C800058EC2AF0B2EC45F0FF0E58EC2AF0C2ECFA
:102C900046F0FF0E58EC2AF092EC46F0FF0E58EC8E
:102CA0002AF022EC47F0000E58EC2AF022EC47F014
:102CB000000E58EC2AF03FB662EF16F03F86115036
:102CC0004A6E4B6E57EC31F01DEC2AF0400E26ECAC
:102CD0002AF0BD0E3FEC2AF04050A9EC38F0F2EC9F
:102CE00038F03F8274EF20F0B8EC3BF03FB27BEF5E
:102CF00016F0070E496E3FA405EC31F01AEC2AF0ED
:102D0000460E26EC2AF0BC0E3FEC2AF0000E495C81
:102D1000D8B4D6EF16F0010E495CD8B4FEEF16F029
:102D2000020E495CD8B426EF17F0030E495CD8B404
:102D300026EF17F0040E495CD8B45AEF17F0050ED1
:102D4000495CD8B45AEF17F0060E495CD8B48EEF40
:102D500017F0080E495CD8B4B4EF17F0FF0E58EC2A
:102D60002AF0A2EC45F0FF0E58EC2AF0F2EC45F008
:102D7000FF0E58EC2AF0A2EC46F0FF0E58EC2AF0B9
:102D800022EC47F0000E58EC2AF022EC47F0000E3F
:102D900058EC2AF022EC47F0000E58EC2AF022EC16
:102DA00047F0000E58EC2AF0B4EF17F0FF0E58EC85
:102DB0002AF0A2EC46F0FF0E58EC2AF0E2EC46F0C6
:102DC000FF0E58EC2AF0A2EC45F0FF0E58EC2AF06A
:102DD00032EC46F0FF0E58EC2AF022EC46F0FF0EE3
:102DE00058EC2AF022EC47F0000E58EC2AF022ECC6
:102DF00047F0000E58EC2AF0B4EF17F0FF0E58EC35
:102E00002AF042EC46F0FF0E58EC2AF0C2EC46F0F5
:102E1000FF0E58EC2AF0B2EC46F0FF0E58EC2AF008
:102E2000C2EC45F0FF0E58EC2AF0A2EC46F0FF0E83
:102E300058EC2AF082EC45F0FF0E58EC2AF062ECD8
:102E400046F0FF0E58EC2AF0B4EF17F0FF0E58ECE6
:102E50002AF002EC46F0FF0E58EC2AF052EC46F055
:102E6000FF0E58EC2AF0B2EC46F0FF0E58EC2AF0B8
:102E7000020E495CD8B444EF17F0B2EC41F0FF0EFB
:102E800058EC2AF049EF17F0C2EC41F0FF0E58EC75
:102E90002AF022EC47F0000E58EC2AF022EC47F022
:102EA000000E58EC2AF022EC47F0000E58EC2AF005
:102EB000B4EF17F0FF0E58EC2AF0F2EC45F0FF0EDD
:102EC00058EC2AF062EC46F0FF0E58EC2AF032EC97
:102ED00046F0FF0E58EC2AF0B2EC45F0FF0E58EC2D
:102EE0002AF0040E495CD8B47DEF17F0B2EC41F043
:102EF000FF0E58EC2AF082EF17F0C2EC41F0FF0E03
:102F000058EC2AF022EC47F0000E58EC2AF022ECA4
:102F100047F0000E58EC2AF0B4EF17F0FF0E58EC13
:102F20002AF092EC46F0FF0E58EC2AF042EC46F004
:102F3000FF0E58EC2AF0A2EC45F0FF0E58EC2AF0F8
:102F400022EC46F0FF0E58EC2AF0D2EC45F0FF0ED2
:102F500058EC2AF022EC47F0000E58EC2AF022EC54
:102F600047F0000E58EC2AF03FB6BBEF17F03F8653
:102F700012504A6E4B6E57EC31F01DEC2AF0400EA9
:102F800026EC2AF0BD0E3FEC2AF04050A9EC38F0B8
:102F9000F2EC38F03F8274EF20F011EC3CF03FB2DD
:102FA000D4EF17F0070E496E3FA405EC31F01AEC90
:102FB0002AF0460E26EC2AF0BC0E3FEC2AF0000E5A
:102FC000495CD8B44EEF18F0010E495CD8B480EFDC
:102FD00018F0020E495CD8B480EF18F0030E495C7B
:102FE000D8B480EF18F0080E495CD8B4C8EF18F0D8
:102FF000FF0E58EC2AF0E2EC45F0FF0E58EC2AF0F8
:1030000072EC46F0FF0E58EC2AF062EC46F0FF0E30
:1030100058EC2AF0B2EC41F0FF0E58EC2AF0A2EC8A
:1030200046F0FF0E58EC2AF0C2EC45F0FF0E58ECCB
:103030002AF032EC46F0FF0E58EC2AF0040E495C00
:10304000D8B434EF18F0050E495CD8B43BEF18F053
:10305000060E495CD8B442EF18F0B2EC41F0FF0E16
:1030600058EC2AF047EF18F0E2EC41F0FF0E58EC74
:103070002AF047EF18F0D2EC41F0FF0E58EC2AF09E
:1030800047EF18F0C2EC41F0FF0E58EC2AF022ECAA
:1030900047F0000E58EC2AF0C8EF18F0FF0E58EC7D
:1030A0002AF0B2EC45F0FF0E58EC2AF0C2EC45F0E5
:1030B000FF0E58EC2AF0B2EC46F0FF0E58EC2AF066
:1030C000A2EC45F0FF0E58EC2AF002EC46F0FF0EA1
:1030D00058EC2AF022EC47F0000E58EC2AF022ECD3
:1030E00047F0000E58EC2AF022EC47F0000E58ECA6
:1030F0002AF022EC47F0000E58EC2AF0C8EF18F046
:10310000FF0E58EC2AF0C2EC45F0FF0E58EC2AF006
:1031100042EC46F0FF0E58EC2AF072EC46F0FF0E3F
:1031200058EC2AF0F2EC45F0FF0E58EC2AF0A2EC35
:1031300045F0FF0E58EC2AF052EC46F0FF0E58EC2A
:103140002AF0B2EC46F0FF0E58EC2AF032EC46F0D2
:10315000FF0E58EC2AF0010E495CD8B4BCEF18F011
:10316000020E495CD8B4C3EF18F0B2EC41F0FF0E88
:1031700058EC2AF0C8EF18F0D2EC41F0FF0E58ECF2
:103180002AF0C8EF18F0C2EC41F0FF0E58EC2AF01C
:103190003FB6CFEF18F03F8613504A6E4B6E57EC98
:1031A00031F01DEC2AF0400E26EC2AF0BD0E3FEC6B
:1031B0002AF04050A9EC38F0F2EC38F03F8274EF7E
:1031C00020F06AEC3CF03FB2E8EF18F0070E496ED1
:1031D0003FA405EC31F01AEC2AF0460E26EC2AF05A
:1031E000BC0E3FEC2AF0000E495CD8B45DEF19F03C
:1031F000010E495CD8B45DEF19F0020E495CD8B4F9
:103200005DEF19F0030E495CD8B45DEF19F0080EBC
:10321000495CD8B4ACEF19F0FF0E58EC2AF0E2ECA0
:1032200045F0FF0E58EC2AF072EC46F0FF0E58EC19
:103230002AF062EC46F0FF0E58EC2AF0D2EC41F096
:10324000FF0E58EC2AF0A2EC46F0FF0E58EC2AF0E4
:10325000C2EC45F0FF0E58EC2AF032EC46F0FF0EBF
:1032600058EC2AF0040E495CD8B448EF19F0050E6A
:10327000495CD8B44FEF19F0060E495CD8B456EF4C
:1032800019F0B2EC41F0FF0E58EC2AF0ACEF19F057
:10329000E2EC41F0FF0E58EC2AF0ACEF19F0D2EC62
:1032A00041F0FF0E58EC2AF0ACEF19F0C2EC41F0FF
:1032B000FF0E58EC2AF0ACEF19F0FF0E58EC2AF094
:1032C000E2EC45F0FF0E58EC2AF072EC46F0FF0EEF
:1032D00058EC2AF062EC46F0FF0E58EC2AF0C2ECF3
:1032E00041F0FF0E58EC2AF0A2EC46F0FF0E58EC2D
:1032F0002AF0C2EC45F0FF0E58EC2AF032EC46F012
:10330000FF0E58EC2AF0000E495CD8B499EF19F082
:10331000010E495CD8B4A0EF19F0020E495CD8B494
:10332000A7EF19F0B2EC41F0FF0E58EC2AF0ACEF29
:1033300019F0E2EC41F0FF0E58EC2AF0ACEF19F076
:10334000D2EC41F0FF0E58EC2AF0ACEF19F0C2ECD1
:1033500041F0FF0E58EC2AF03FB6B3EF19F03F866C
:1033600014504A6E4B6E57EC31F01DEC2AF0400EB3
:1033700026EC2AF0BD0E3FEC2AF04050A9EC38F0C4
:10338000F2EC38F03F8274EF20F0C3EC3CF03FB237
:10339000CCEF19F0070E496E3FA405EC31F01AECA2
:1033A0002AF0460E26EC2AF0BC0E3FEC2AF0000E66
:1033B000495CD8B401EF1AF0010E495CD8B424EF8F
:1033C0001AF0020E495CD8B447EF1AF0030E495CBC
:1033D000D8B447EF1AF0040E495CD8B447EF1AF09E
:1033E000050E495CD8B482EF1AF0060E495CD8B4D9
:1033F00082EF1AF0080E495CD8B4BBEF1AF082EFE6
:103400001AF0FF0E58EC2AF092EC46F0FF0E58EC42
:103410002AF0C2EC46F0FF0E58EC2AF052EC46F0CF
:10342000FF0E58EC2AF022EC47F0000E58EC2AF080
:1034300022EC47F0000E58EC2AF022EC47F0000E88
:1034400058EC2AF0BBEF1AF0FF0E58EC2AF092EC81
:1034500046F0FF0E58EC2AF0F2EC46F0FF0E58EC66
:103460002AF0B2EC45F0FF0E58EC2AF022EC47F0BF
:10347000000E58EC2AF022EC47F0000E58EC2AF02F
:1034800022EC47F0000E58EC2AF0BBEF1AF0FF0ECA
:1034900058EC2AF092EC46F0FF0E58EC2AF0F2ECD1
:1034A00046F0FF0E58EC2AF0A2EC46F0FF0E58EC66
:1034B0002AF0C2EC45F0FF0E58EC2AF032EC46F050
:1034C000FF0E58EC2AF0020E495CD8B474EF1AF0E3
:1034D000030E495CD8B47BEF1AF0B2EC41F0FF0E5A
:1034E00058EC2AF0BBEF1AF0D2EC41F0FF0E58EC8A
:1034F0002AF0BBEF1AF0C2EC41F0FF0E58EC2AF0B4
:10350000BBEF1AF0FF0E58EC2AF0B2EC46F0FF0EBB
:1035100058EC2AF0F2EC46F0FF0E58EC2AF0A2EC40
:1035200046F0FF0E58EC2AF0C2EC45F0FF0E58ECC6
:103530002AF032EC46F0FF0E58EC2AF0050E495CFA
:10354000D8B4AFEF1AF0060E495CD8B4B6EF1AF053
:10355000B2EC41F0FF0E58EC2AF0BBEF1AF0D2ECBF
:1035600041F0FF0E58EC2AF0BBEF1AF0C2EC41F02C
:10357000FF0E58EC2AF03FB6C2EF1AF03F86155006
:103580004A6E4B6E57EC31F01DEC2AF0400E26ECE3
:103590002AF0BD0E3FEC2AF04050A9EC38F0F2ECD6
:1035A00038F03F8274EF20F01CEC3DF03FB2DBEFCF
:1035B0001AF0070E496E3FA405EC31F01AEC2AF020
:1035C000460E26EC2AF0BC0E3FEC2AF0080E495CB1
:1035D000D8B4E2EF1BF0FF0E58EC2AF0A2EC46F054
:1035E000FF0E58EC2AF062EC46F0FF0E58EC2AF081
:1035F000000E495CD8B436EF1BF0010E495CD8B41C
:1036000051EF1BF0020E495CD8B46CEF1BF0030EB7
:10361000495CD8B46CEF1BF0040E495CD8B493EF4E
:103620001BF0050E495CD8B4AEEF1BF0060E495CEA
:10363000D8B4C9EF1BF032EC46F0FF0E58EC2AF07C
:1036400092EC46F0FF0E58EC2AF072EC46F0FF0EBA
:1036500058EC2AF062EC46F0FF0E58EC2AF032ECFF
:1036600046F0FF0E58EC2AF0E2EF1BF042EC46F079
:10367000FF0E58EC2AF0A2EC46F0FF0E58EC2AF0B0
:1036800022EC47F0000E58EC2AF022EC47F0000E36
:1036900058EC2AF022EC47F0000E58EC2AF0E2EF4A
:1036A0001BF0A2EC46F0FF0E58EC2AF0D2EC45F0ED
:1036B000FF0E58EC2AF022EC47F0000E58EC2AF0EE
:1036C00022EC47F0000E58EC2AF022EC47F0000EF6
:1036D00058EC2AF0E2EF1BF092EC46F0FF0E58ECAB
:1036E0002AF0C2EC45F0FF0E58EC2AF0A2EC46F0AE
:1036F000FF0E58EC2AF0020E495CD8B487EF1BF09D
:10370000B2EC41F0FF0E58EC2AF08CEF1BF0C2EC4B
:1037100041F0FF0E58EC2AF022EC47F0000E58EC76
:103720002AF0E2EF1BF012EC46F0FF0E58EC2AF004
:10373000C2EC46F0FF0E58EC2AF0A2EC46F0FF0E69
:1037400058EC2AF0B2EC46F0FF0E58EC2AF022ECCE
:1037500047F0000E58EC2AF0E2EF1BF0B2EC45F017
:10376000FF0E58EC2AF0C2EC45F0FF0E58EC2AF0A0
:1037700032EC46F0FF0E58EC2AF022EC47F0000E37
:1037800058EC2AF022EC47F0000E58EC2AF0E2EF59
:103790001BF0A2EC46F0FF0E58EC2AF072EC46F05B
:1037A000FF0E58EC2AF062EC46F0FF0E58EC2AF0BF
:1037B00032EC46F0FF0E58EC2AF022EC47F0000EF7
:1037C00058EC2AF03FB6E9EF1BF03F8616504A6EE0
:1037D0004B6E57EC31F01DEC2AF0400E26EC2AF02F
:1037E000BD0E3FEC2AF04050A9EC38F0F2EC38F076
:1037F0003F8274EF20F0C5EC3DF03FB202EF1CF0C9
:10380000070E496E3FA42EEC31F01AEC2AF0460E5A
:1038100026EC2AF0BC0E3FEC2AF0010E495CD8B42D
:1038200058EF1CF0020E495CD8B480EF1CF0030E78
:10383000495CD8B4A8EF1CF0040E495CD8B4D0EFB2
:103840001CF0050E495CD8B4F8EF1CF0060E495C7C
:10385000D8B420EF1DF0080E495CD8B446EF1DF037
:10386000FF0E58EC2AF072EC46F0FF0E58EC2AF0EE
:1038700082EC45F0FF0E58EC2AF092EC46F0FF0E79
:1038800058EC2AF042EC46F0FF0E58EC2AF022ECFD
:1038900047F0000E58EC2AF022EC47F0000E58ECEE
:1038A0002AF022EC47F0000E58EC2AF046EF1DF00B
:1038B000FF0E58EC2AF082EC46F0FF0E58EC2AF08E
:1038C000A2EC45F0FF0E58EC2AF092EC46F0FF0E09
:1038D00058EC2AF0A2EC45F0FF0E58EC2AF042EC2E
:1038E00046F0FF0E58EC2AF022EC47F0000E58ECA0
:1038F0002AF022EC47F0000E58EC2AF046EF1DF0BB
:10390000FF0E58EC2AF0A2EC45F0FF0E58EC2AF01E
:10391000A2EC45F0FF0E58EC2AF092EC46F0FF0EB8
:1039200058EC2AF0A2EC45F0FF0E58EC2AF042ECDD
:1039300046F0FF0E58EC2AF022EC47F0000E58EC4F
:103940002AF022EC47F0000E58EC2AF046EF1DF06A
:10395000FF0E58EC2AF0C2EC46F0FF0E58EC2AF0AD
:1039600052EC46F0FF0E58EC2AF032EC46F0FF0E17
:1039700058EC2AF062EC46F0FF0E58EC2AF0A2EC6C
:1039800045F0FF0E58EC2AF022EC46F0FF0E58EC02
:103990002AF042EC46F0FF0E58EC2AF046EF1DF0FC
:1039A000FF0E58EC2AF0D2EC46F0FF0E58EC2AF04D
:1039B00042EC46F0FF0E58EC2AF022EC47F0000EE5
:1039C00058EC2AF022EC47F0000E58EC2AF022ECDA
:1039D00047F0000E58EC2AF022EC47F0000E58ECAD
:1039E0002AF022EC47F0000E58EC2AF046EF1DF0CA
:1039F000FF0E58EC2AF0A2EC45F0FF0E58EC2AF02E
:103A000062EC46F0FF0E58EC2AF042EC46F0FF0E56
:103A100058EC2AF0D2EC45F0FF0E58EC2AF042ECBC
:103A200046F0FF0E58EC2AF022EC47F0000E58EC5E
:103A30002AF022EC47F0000E58EC2AF046EF1DF079
:103A4000FF0E58EC2AF092EC45F0FF0E58EC2AF0ED
:103A500002EC46F0FF0E58EC2AF072EC46F0FF0E36
:103A600058EC2AF042EC46F0FF0E58EC2AF022EC1B
:103A700047F0000E58EC2AF022EC47F0000E58EC0C
:103A80002AF022EC47F0000E58EC2AF03FB64DEF3A
:103A90001DF03F8617504A6E4B6E57EC31F01DEC0F
:103AA0002AF0400E26EC2AF0BD0E3FEC2AF04050E2
:103AB000A9EC38F0F2EC38F03F8274EF20F053ECD0
:103AC0003EF03FB266EF1DF0070E496E3FA42EECAC
:103AD00031F01AEC2AF0460E26EC2AF0BC0E3FEC30
:103AE0002AF0010E495CD8B4A7EF1DF0020E495C24
:103AF000D8B4B5EF1DF0030E495CD8B4BEEF1DF08D
:103B0000040E495CD8B4CCEF1DF0050E495CD8B466
:103B1000DFEF1DF0060E495CD8B4EDEF1DF0080E86
:103B2000495CD8B4FEEF1DF05FEC40F042EC46F08B
:103B3000FF0E58EC2AF022EC47F0000E58EC2AF069
:103B400022EC47F0000E58EC2AF0FEEF1DF0D4EC0A
:103B50003FF042EC46F0FF0E58EC2AF022EC47F022
:103B6000000E58EC2AF0FEEF1DF0ECEC3FF042ECBA
:103B700046F0FF0E58EC2AF0FEEF1DF009EC40F085
:103B800042EC46F0FF0E58EC2AF022EC47F0000E13
:103B900058EC2AF0FEEF1DF021EC40F042EC46F02C
:103BA000FF0E58EC2AF022EC47F0000E58EC2AF0F9
:103BB00022EC47F0000E58EC2AF0FEEF1DF034EC3A
:103BC00040F042EC46F0FF0E58EC2AF022EC47F0B1
:103BD000000E58EC2AF0FEEF1DF04CEC40F042ECE9
:103BE00046F0FF0E58EC2AF022EC47F0000E58EC9D
:103BF0002AF022EC47F0000E58EC2AF03FB605EF11
:103C00001EF03F8618504A6E4B6E57EC31F01DEC9B
:103C10002AF0400E26EC2AF0BD0E3FEC2AF0405070
:103C2000A9EC38F0F2EC38F03F8274EF20F0C2ECEF
:103C30003EF03FB21EEF1EF0070E496E3FA42EEC81
:103C400031F01AEC2AF0460E26EC2AF0BC0E3FECBE
:103C50002AF0010E495CD8B45FEF1EF0020E495CF9
:103C6000D8B46DEF1EF0030E495CD8B476EF1EF0A9
:103C7000040E495CD8B484EF1EF0050E495CD8B43C
:103C800097EF1EF0060E495CD8B4A5EF1EF0080EA3
:103C9000495CD8B4B6EF1EF05FEC40F0C2EC41F0E6
:103CA000FF0E58EC2AF022EC47F0000E58EC2AF0F8
:103CB00022EC47F0000E58EC2AF0B6EF1EF0D4ECE0
:103CC0003FF0C2EC41F0FF0E58EC2AF022EC47F036
:103CD000000E58EC2AF0B6EF1EF0ECEC3FF0C2EC10
:103CE00041F0FF0E58EC2AF0B6EF1EF009EC40F060
:103CF000C2EC41F0FF0E58EC2AF022EC47F0000E27
:103D000058EC2AF0B6EF1EF021EC40F0C2EC41F086
:103D1000FF0E58EC2AF022EC47F0000E58EC2AF087
:103D200022EC47F0000E58EC2AF0B6EF1EF034EC0F
:103D300040F0C2EC41F0FF0E58EC2AF022EC47F0C4
:103D4000000E58EC2AF0B6EF1EF04CEC40F0C2EC3E
:103D500041F0FF0E58EC2AF022EC47F0000E58EC30
:103D60002AF022EC47F0000E58EC2AF03FB6BDEFE7
:103D70001EF03F8619504A6E4B6E57EC31F01DEC29
:103D80002AF0400E26EC2AF0BD0E3FEC2AF04050FF
:103D9000A9EC38F0F2EC38F03F8274EF20F04BECF5
:103DA0003FF03FB2D6EF1EF0070E496E3FA42EEC57
:103DB00031F01AEC2AF0460E26EC2AF0BC0E3FEC4D
:103DC0002AF0010E495CD8B417EF1FF0020E495CCF
:103DD000D8B425EF1FF0030E495CD8B42EEF1FF0C6
:103DE000040E495CD8B43CEF1FF0050E495CD8B412
:103DF0004FEF1FF0060E495CD8B45DEF1FF0080EC0
:103E0000495CD8B46EEF1FF05FEC40F0B2EC41F0CB
:103E1000FF0E58EC2AF022EC47F0000E58EC2AF086
:103E200022EC47F0000E58EC2AF06EEF1FF0D4ECB5
:103E30003FF0B2EC41F0FF0E58EC2AF022EC47F0D4
:103E4000000E58EC2AF06EEF1FF0ECEC3FF0B2ECF5
:103E500041F0FF0E58EC2AF06EEF1FF009EC40F035
:103E6000B2EC41F0FF0E58EC2AF022EC47F0000EC5
:103E700058EC2AF06EEF1FF021EC40F0B2EC41F06C
:103E8000FF0E58EC2AF022EC47F0000E58EC2AF016
:103E900022EC47F0000E58EC2AF06EEF1FF034ECE5
:103EA00040F0B2EC41F0FF0E58EC2AF022EC47F063
:103EB000000E58EC2AF06EEF1FF04CEC40F0B2EC24
:103EC00041F0FF0E58EC2AF022EC47F0000E58ECBF
:103ED0002AF022EC47F0000E58EC2AF03FB675EFBE
:103EE0001FF03F861A504A6E4B6E57EC31F01DECB6
:103EF0002AF0400E26EC2AF0BD0E3FEC2AF040508E
:103F0000A9EC38F0F2EC38F03F8274EF20F022ECAC
:103F100044F0000E58EC2AF032EC44F0000E58EC5D
:103F20002AF042EC44F0000E58EC2AF0F2EC43F098
:103F3000000E58EC2AF022EC45F0000E58EC2AF066
:103F400092EC44F0000E58EC2AF012EC45F0000E12
:103F500058EC2AF022EC47F092EC44F0000E58ECBA
:103F60002AF0C2EC44F01DEC2AF0400E26EC2AF0B8
:103F7000B90E3FEC2AF0000E58EC2AF0F2EC43F0B8
:103F8000000E58EC2AF022EC44F0000E58EC2AF017
:103F90001AEC2AF0670E26EC2AF0BC0E3FEC2AF051
:103FA0003FB0E7EF1FF0000E58EC2AF062EC45F04E
:103FB000000E58EC2AF032EC44F0000E58EC2AF0D7
:103FC00002EC45F0000E58EC2AF0F9EF1FF0FF0E5E
:103FD00058EC2AF002EC47F0FF0E58EC2AF0C2EC45
:103FE00045F0FF0E58EC2AF0A2EC46F0FF0E58EC1C
:103FF0002AF01DEC2AF0440E26EC2AF0BC0E3FEC11
:104000002AF03FB018EF20F0FF0E58EC2AF052ECE7
:1040100046F0FF0E58EC2AF032EC47F0FF0E58EC59
:104020002AF062EC46F0FF0E58EC2AF02AEF20F05E
:10403000000E58EC2AF0B2EC44F0000E58EC2AF0D6
:1040400022EC47F0000E58EC2AF0C2EC44F0000ECF
:1040500058EC2AF080B03AEF20F03EB03BEF20F071
:104060003FB036EF20F03F8037EF20F03F903E80AA
:104070003BEF20F03E9084B64BEF20F03EBC4CEF7F
:1040800020F03FB047EF20F03F8048EF20F03F9016
:104090003E8C4CEF20F03E9C80B873EF20F03EB891
:1040A00074EF20F0436A466A42EC2BF03FA06FEFBA
:1040B00020F0080E116E040E126E4B0E136EBB0E26
:1040C000146E9B0E156E880E166E7F0E176E7F0E89
:1040D000186E000E196E000E1A6E5FEC2BF03F90FA
:1040E0003E881BEF01F03E9880BA87EF20F03EBA81
:1040F0001BEF01F0000E436E3E8A466A42EC2BF045
:104100003F903F923F96496A4A6A1BEF01F03E9A00
:104110001BEF01F01AEC2AF0410E26EC2AF0B80E43
:104120003FEC2AF0700E58EC2AF0100E58EC2AF0F2
:10413000100E58EC2AF0100E58EC2AF0000E58EC35
:104140002AF032EC44F0000E58EC2AF032EC44F045
:10415000000E58EC2AF0D2EC44F0000E58EC2AF095
:10416000F2EC44F0000E58EC2AF0C2EC44F0000EE1
:1041700058EC2AF0A2EC44F0000E58EC2AF022ECA5
:1041800047F042EC45F0000E58EC2AF0F2EC44F017
:10419000000E58EC2AF072EC44F01DEC2AF0400EB0
:1041A00026EC2AF0B80E3FEC2AF0000E58EC2AF06C
:1041B00012EC45F0000E58EC2AF032EC44F0000E00
:1041C00058EC2AF0082A320E085CD8B4EDEF20F043
:1041D000100E58EC2AF0E2EF20F0086A700E58EC4E
:1041E0002AF0000E445CD8B4FDEF20F0010E445CD0
:1041F000D8B487EF24F01BEF01F01AEC2AF0460E3A
:1042000026EC2AF0B90E3FEC2AF002EC45F0000E45
:1042100058EC2AF032EC44F0000E58EC2AF092EC04
:1042200044F0000E58EC2AF032EC44F0000E58EC4A
:104230002AF012EC44F0000E58EC2AF012EC45F093
:10424000000E58EC2AF022EC47F0F2EC43F0000E9E
:1042500058EC2AF022EC44F0000E58EC2AF022EC44
:1042600044F01DEC2AF0400E26EC2AF0B90E3FEC8B
:104270002AF0000E58EC2AF0F2EC44F0000E58EC54
:104280002AF032EC44F0000E58EC2AF002EC45F033
:10429000000E58EC2AF002EC45F0000E58EC2AF023
:1042A00080B062EF21F03EB063EF21F00B0E475C6F
:1042B000D8B45EEF21F0472A5FEF21F0476A3E80D5
:1042C00063EF21F03E9084B676EF21F03EBC77EFAD
:1042D00021F0000E475CD8B471EF21F0470673EF70
:1042E00021F00B0E476E3E8C77EF21F03E9C1AECCE
:1042F0002AF04A0E26EC2AF0BB0E3FEC2AF0000E04
:10430000475CD8B498EF21F0000E58EC2AF012EC7C
:1043100041F0000E58EC2AF012EC41F0000E58EC7F
:104320002AF062EC44F0000E58EC2AF0AAEF21F0DB
:10433000FF0E58EC2AF0B2EC41F0FF0E58EC2AF0D8
:10434000B2EC41F0FF0E58EC2AF0F2EC45F0FF0E13
:1043500058EC2AF01AEC2AF0670E26EC2AF0BB0E75
:104360003FEC2AF0010E475CD8B4CBEF21F0000EF1
:1043700058EC2AF012EC41F0000E58EC2AF022EC36
:1043800041F0000E58EC2AF062EC44F0000E58ECBC
:104390002AF0DDEF21F0FF0E58EC2AF0B2EC41F0EC
:1043A000FF0E58EC2AF0C2EC41F0FF0E58EC2AF058
:1043B000F2EC45F0FF0E58EC2AF01DEC2AF0440E0A
:1043C00026EC2AF0BB0E3FEC2AF0020E475CD8B474
:1043D000FEEF21F0000E58EC2AF012EC41F0000E36
:1043E00058EC2AF032EC41F0000E58EC2AF062EC66
:1043F00044F0000E58EC2AF010EF22F0FF0E58ECBB
:104400002AF0B2EC41F0FF0E58EC2AF0D2EC41F069
:10441000FF0E58EC2AF0F2EC45F0FF0E58EC2AF0B3
:104420001DEC2AF0610E26EC2AF0BB0E3FEC2AF0C0
:10443000030E475CD8B431EF22F0000E58EC2AF09E
:1044400012EC41F0000E58EC2AF042EC41F0000E64
:1044500058EC2AF062EC44F0000E58EC2AF043EFDE
:1044600022F0FF0E58EC2AF0B2EC41F0FF0E58ECAF
:104470002AF0E2EC41F0FF0E58EC2AF0F2EC45F0A5
:10448000FF0E58EC2AF01AEC2AF04A0E26EC2AF01D
:10449000BC0E3FEC2AF0040E475CD8B464EF22F067
:1044A000000E58EC2AF012EC41F0000E58EC2AF005
:1044B00052EC41F0000E58EC2AF062EC44F0000E91
:1044C00058EC2AF076EF22F0FF0E58EC2AF0B2EC0E
:1044D00041F0FF0E58EC2AF0F2EC41F0FF0E58ECE0
:1044E0002AF0F2EC45F0FF0E58EC2AF01AEC2AF014
:1044F000670E26EC2AF0BC0E3FEC2AF0050E475C56
:10450000D8B497EF22F0000E58EC2AF012EC41F0EC
:10451000000E58EC2AF062EC41F0000E58EC2AF044
:1045200062EC44F0000E58EC2AF0A9EF22F0FF0EE6
:1045300058EC2AF0B2EC41F0FF0E58EC2AF002ECF5
:1045400042F0FF0E58EC2AF0F2EC45F0FF0E58EC6A
:104550002AF01DEC2AF0440E26EC2AF0BC0E3FECAB
:104560002AF0060E475CD8B4CAEF22F0000E58ECD1
:104570002AF012EC41F0000E58EC2AF072EC41F0F7
:10458000000E58EC2AF062EC44F0000E58EC2AF0D1
:10459000DCEF22F0FF0E58EC2AF0B2EC41F0FF0EF7
:1045A00058EC2AF012EC42F0FF0E58EC2AF0F2EC34
:1045B00045F0FF0E58EC2AF01DEC2AF0610E26ECB7
:1045C0002AF0B40E3FEC2AF0070E475CD8B4FDEF9A
:1045D00022F0000E58EC2AF012EC41F0000E58ECDC
:1045E0002AF082EC41F0000E58EC2AF062EC44F024
:1045F000000E58EC2AF00FEF23F0FF0E58EC2AF0D3
:10460000B2EC41F0FF0E58EC2AF022EC42F0FF0E23
:1046100058EC2AF0F2EC45F0FF0E58EC2AF01AECB8
:104620002AF04A0E26EC2AF0BD0E3FEC2AF0080EC6
:10463000475CD8B430EF23F0000E58EC2AF012ECAF
:1046400041F0000E58EC2AF092EC41F0000E58ECCC
:104650002AF062EC44F0000E58EC2AF042EF23F00E
:10466000FF0E58EC2AF0B2EC41F0FF0E58EC2AF0A5
:1046700032EC42F0FF0E58EC2AF0F2EC45F0FF0E5F
:1046800058EC2AF01AEC2AF0670E26EC2AF0BD0E40
:104690003FEC2AF0090E475CD8B463EF23F0000E1C
:1046A00058EC2AF012EC41F0000E58EC2AF0A2EC83
:1046B00041F0000E58EC2AF062EC44F0000E58EC89
:1046C0002AF075EF23F0FF0E58EC2AF0B2EC41F01F
:1046D000FF0E58EC2AF042EC42F0FF0E58EC2AF0A4
:1046E000F2EC45F0FF0E58EC2AF01AEC2AF04A0ED4
:1046F00026EC2AF0BE0E3FEC2AF00A0E475CD8B436
:10470000B1EF23F0000E58EC2AF0C2EC44F0000E9A
:1047100058EC2AF012EC45F0000E58EC2AF062EC4E
:1047200044F0000E58EC2AF032EC44F0000E58EC45
:104730002AF0F2EC44F0000E58EC2AF022EC47F09C
:1047400002EC45F0000E58EC2AF032EC44F0000E7A
:1047500058EC2AF012EC45F0000E58EC2AF0DEEF8F
:1047600023F0FF0E58EC2AF062EC46F0FF0E58ECF6
:104770002AF0B2EC46F0FF0E58EC2AF0F2EC45F0CD
:10478000FF0E58EC2AF0C2EC45F0FF0E58EC2AF070
:1047900092EC46F0FF0E58EC2AF032EC47F0A2EC17
:1047A00046F0FF0E58EC2AF0C2EC45F0FF0E58EC34
:1047B0002AF0B2EC46F0FF0E58EC2AF01AEC2AF080
:1047C0004A0E26EC2AF0BF0E3FEC2AF00B0E475C97
:1047D000D8B431EF24F0000E58EC2AF0F2EC43F09C
:1047E000000E58EC2AF092EC44F0000E58EC2AF03F
:1047F00092EC44F0000E58EC2AF022EC47F0F2EC78
:1048000044F0000E58EC2AF032EC44F0000E58EC64
:104810002AF052EC44F0000E58EC2AF072EC44F00E
:10482000000E58EC2AF002EC45F0000E58EC2AF08D
:104830001DEC2AF0400E26EC2AF0BF0E3FEC2AF0C9
:1048400012EC45F0000E58EC2AF032EC44F0000E69
:1048500058EC2AF0F2EC44F0000E58EC2AF075EF18
:1048600024F0FF0E58EC2AF082EC45F0FF0E58ECD5
:104870002AF032EC46F0FF0E58EC2AF032EC46F00B
:10488000FF0E58EC2AF032EC47F092EC46F0FF0EA7
:1048900058EC2AF0C2EC45F0FF0E58EC2AF0E2EC9E
:1048A00045F0FF0E58EC2AF002EC46F0FF0E58ECF3
:1048B0002AF0A2EC46F0FF0E58EC2AF01DEC2AF08C
:1048C000400E26EC2AF0BF0E3FEC2AF0B2EC46F088
:1048D000FF0E58EC2AF0C2EC45F0FF0E58EC2AF01F
:1048E00092EC46F0FF0E58EC2AF0DBEC2DF080B88D
:1048F00084EF24F03EB885EF24F0010E446E42ECC4
:104900002BF03E8885EF24F03E981BEF01F01AEC67
:104910002AF0460E26EC2AF0B90E3FEC2AF0000EE3
:10492000475CD8B4C8EF24F0010E475CD8B4D0EF90
:1049300024F0020E475CD8B4D8EF24F0030E475C95
:10494000D8B4E0EF24F0040E475CD8B4E8EF24F0CC
:10495000050E475CD8B4F0EF24F0060E475CD8B4DF
:10496000F8EF24F0070E475CD8B400EF25F0080EEE
:10497000475CD8B408EF25F0090E475CD8B410EFB7
:1049800025F00A0E475CD8B418EF25F072EF25F039
:104990005FEC3BF0AEEC33F033EC34F0F9EF25F0A4
:1049A000B8EC3BF0AEEC33F033EC34F0F9EF25F03B
:1049B00011EC3CF0AEEC33F033EC34F0F9EF25F0D1
:1049C0006AEC3CF0AEEC33F033EC34F0F9EF25F068
:1049D000C3EC3CF0AEEC33F033EC34F0F9EF25F0FF
:1049E0001CEC3DF0AEEC33F033EC34F0F9EF25F095
:1049F000C5EC3DF0AEEC33F033EC34F0F9EF25F0DC
:104A000053EC3EF0AEEC33F033EC34F0F9EF25F03C
:104A1000C2EC3EF0AEEC33F033EC34F0F9EF25F0BD
:104A20004BEC3FF0AEEC33F033EC34F0F9EF25F023
:104A3000000E58EC2AF0C2EC44F0000E58EC2AF0BC
:104A400012EC45F0000E58EC2AF062EC44F0000E37
:104A500058EC2AF032EC44F0000E58EC2AF0F2EC5C
:104A600044F0000E58EC2AF022EC47F002EC45F03E
:104A7000000E58EC2AF032EC44F0000E58EC2AF00C
:104A800012EC45F0000E58EC2AF01DEC2AF0400E16
:104A900026EC2AF0B90E3FEC2AF0000E58EC2AF072
:104AA000000E58EC2AF042EC45F0000E58EC2AF0CB
:104AB000F2EC44F0000E58EC2AF072EC44F0000ED8
:104AC00058EC2AF012EC45F0000E58EC2AF032ECCB
:104AD00044F0000E58EC2AF0AEEC33F033EC34F036
:104AE000F9EF25F0F2EC43F0000E58EC2AF092ECCE
:104AF00044F0000E58EC2AF092EC44F0000E58EC12
:104B00002AF022EC47F0F2EC44F0000E58EC2AF0C8
:104B100032EC44F0000E58EC2AF052EC44F0000E57
:104B200058EC2AF072EC44F0000E58EC2AF002EC3B
:104B300045F0000E58EC2AF012EC45F01DEC2AF07E
:104B4000400E26EC2AF0B90E3FEC2AF0000E58EC8D
:104B50002AF032EC44F0000E58EC2AF0F2EC44F06B
:104B6000000E58EC2AF022EC47F042EC45F0000E23
:104B700058EC2AF0F2EC44F0000E58EC2AF072ECFB
:104B800044F0000E58EC2AF012EC45F0000E58EC00
:104B90002AF032EC44F0000E58EC2AF0AEEC33F080
:104BA00080B8F8EF25F03EB8F9EF25F03FACF1EF13
:104BB00025F042EC2BF05AEC47F06DEC47F080EC1E
:104BC00047F093EC47F0A6EC47F0B9EC47F0CCEC9B
:104BD00047F0DFEC47F0F2EC47F005EC48F018EC5A
:104BE00048F0446A476A3F9C3F903E881BEF01F0C3
:104BF0003E9880BA1BEF01F0000E446E3E8A476A71
:104C000042EC2BF03F9C1BEF01F01AEC2AF0410E16
:104C100026EC2AF0B80E3FEC2AF0700E58EC2AF081
:104C2000100E58EC2AF0100E58EC2AF0100E58EC2A
:104C30002AF0000E58EC2AF0C2EC44F0000E58ECBA
:104C40002AF012EC45F0000E58EC2AF062EC44F029
:104C5000000E58EC2AF032EC44F0000E58EC2AF02A
:104C6000F2EC44F0000E58EC2AF022EC47F002EC93
:104C700045F0000E58EC2AF032EC44F0000E58ECEF
:104C80002AF012EC45F0000E58EC2AF012EC45F038
:104C90001DEC2AF0400E26EC2AF0B80E3FEC2AF06C
:104CA000000E58EC2AF072EC44F0000E58EC2AF09A
:104CB000B2EC44F0000E58EC2AF052EC44F0000E36
:104CC00058EC2AF0082A2C0E085CD8B46DEF26F0B8
:104CD000100E58EC2AF062EF26F0086A700E58ECBD
:104CE0002AF01AEC2AF0460E26EC2AF0BF0E3FEC12
:104CF0002AF002EC45F0000E58EC2AF0C2EC44F029
:104D0000000E58EC2AF042EC44F0000E58EC2AF069
:104D100012EC45F0000E58EC2AF042EC45F0000E83
:104D200058EC2AF0F2EC43F0000E58EC2AF0F2ECCA
:104D300044F0000E58EC2AF032EC44F0000E58EC2F
:104D40002AF022EC47F032EC45F01DEC2AF0400E40
:104D500026EC2AF0BF0E3FEC2AF0000E58EC2AF0A9
:104D600032EC44F0000E58EC2AF0F2EC44F0000E65
:104D700058EC2AF002EC45F0000E58EC2AF072ECE8
:104D800044F0000E58EC2AF0C2EC44F0000E58EC4F
:104D90002AF0B2EC44F0000E58EC2AF022EC47F076
:104DA000000E58EC2AF022EC41F0000E58EC2AF0EC
:104DB000000E58EC2AF0400E58EC2AF0000E58EC89
:104DC0002AF012EC41F0000E58EC2AF012EC41F0FF
:104DD000000E58EC2AF01AEC2AF0450E26EC2AF0C8
:104DE000BA0E3FEC2AF04CBE37EF27F0000E485CBD
:104DF000D8A437EF27F0FF0E58EC2AF0C2EC45F0AC
:104E0000FF0E58EC2AF092EC46F0FF0E58EC2AF018
:104E100092EC46F0FF0E58EC2AF062EC46F0FF0EE2
:104E200058EC2AF092EC46F0FF0E58EC2AF032ECE7
:104E300047F0F2EC45F0FF0E58EC2AF062EC46F039
:104E4000FF0E58EC2AF032EC46F0FF0E58EC2AF038
:104E5000B2EC45F01DEC2AF0400E26EC2AF0BA0E1A
:104E60003FEC2AF0FF0E58EC2AF071EF27F0000E0D
:104E700058EC2AF032EC44F0000E58EC2AF0F2EC38
:104E800044F0000E58EC2AF0F2EC44F0000E58EC1E
:104E90002AF0C2EC44F0000E58EC2AF0F2EC44F098
:104EA000000E58EC2AF022EC47F062EC44F0000EC1
:104EB00058EC2AF0C2EC44F0000E58EC2AF092ECC8
:104EC00044F0000E58EC2AF022EC44F01DEC2AF0DD
:104ED000400E26EC2AF0BA0E3FEC2AF0000E58ECF9
:104EE0002AF01AEC2AF0450E26EC2AF0BB0E3FEC15
:104EF0002AF04CBEB0EF27F0010E485CD8A4B0EF0A
:104F000027F0FF0E58EC2AF0B2EC46F0FF0E58ECFA
:104F10002AF0F2EC46F0FF0E58EC2AF032EC47F0A3
:104F200062EC46F0FF0E58EC2AF0C2EC46F0FF0EA1
:104F300058EC2AF0B2EC46F0FF0E58EC2AF072EC76
:104F400046F0FF0E58EC2AF0C2EC46F0FF0E58EC8B
:104F50002AF0B2EC46F0FF0E58EC2AF0DDEF27F015
:104F6000000E58EC2AF012EC45F0000E58EC2AF036
:104F700052EC45F0000E58EC2AF022EC47F0C2EC5F
:104F800044F0000E58EC2AF022EC45F0000E58ECEC
:104F90002AF012EC45F0000E58EC2AF0D2EC44F066
:104FA000000E58EC2AF022EC45F0000E58EC2AF0E6
:104FB00012EC45F0000E58EC2AF01AEC2AF0450EDF
:104FC00026EC2AF0BC0E3FEC2AF04CBE29EF28F06C
:104FD000020E485CD8A429EF28F0FF0E58EC2AF006
:104FE000A2EC46F0FF0E58EC2AF0C2EC45F0FF0EA2
:104FF00058EC2AF032EC46F0FF0E58EC2AF0C2ECE6
:1050000045F0FF0E58EC2AF0A2EC45F0FF0E58ECEC
:105010002AF0B2EC46F0FF0E58EC2AF032EC47F0E2
:10502000C2EC46F0FF0E58EC2AF0A2EC46F0FF0E60
:1050300058EC2AF092EC45F01DEC2AF0400E26ECDC
:105040002AF0BC0E3FEC2AF0FF0E58EC2AF063EF7A
:1050500028F0000E58EC2AF002EC45F0000E58EC57
:105060002AF032EC44F0000E58EC2AF092EC44F0B6
:10507000000E58EC2AF032EC44F0000E58EC2AF006
:1050800012EC44F0000E58EC2AF012EC45F0000E41
:1050900058EC2AF022EC47F022EC45F0000E58ECD8
:1050A0002AF002EC45F0000E58EC2AF002EC44F035
:1050B0001DEC2AF0400E26EC2AF0BC0E3FEC2AF044
:1050C000000E58EC2AF04CBE8DEF28F080B078EF3F
:1050D00028F03EB079EF28F0020E485CD8B474EFA7
:1050E00028F0482A75EF28F0486A3E8079EF28F0CA
:1050F0003E9084B68CEF28F03EBC8DEF28F0000E79
:10510000485CD8B487EF28F0480689EF28F0020EF3
:10511000486E3E8C8DEF28F03E9C4CBE9DEF28F0F3
:1051200080B89CEF28F03EB89DEF28F04C8E4C5094
:105130004D6E3E889DEF28F03E984CAEADEF28F0C6
:1051400080BAACEF28F03EBAADEF28F04C9E42ECAE
:105150002BF03E8AADEF28F03E9A4CAEBFEF28F020
:1051600080B8BEEF28F03EB8BFEF28F04D504C6E2F
:105170004C9E42EC2BF03E88BFEF28F03E984CAEA0
:1051800006EF29F080B0E3EF28F03EB0E4EF28F01E
:10519000000E485CD8B4D9EF28F0010E485CD8B4B2
:1051A000DCEF28F0020E485CD8B4DFEF28F0E0EF27
:1051B00028F04D70E0EF28F04D72E0EF28F04D74CC
:1051C0003E80E4EF28F03E9084B605EF29F03EBC27
:1051D00006EF29F0000E485CD8B4FBEF28F0010E72
:1051E000485CD8B4FEEF28F0020E485CD8B401EF5A
:1051F00029F002EF29F04D7002EF29F04D7202EF15
:1052000029F04D743E8C06EF29F03E9C4CAE15EF14
:105210002AF0000E485CD8B41AEF29F0010E485C61
:10522000D8B457EF29F0020E485CD8B4C6EF29F085
:1052300015EF2AF01DEC2AF0460E26EC2AF0BA0EE5
:105240003FEC2AF04DA03EEF29F0FF0E58EC2AF07B
:10525000F2EC45F0FF0E58EC2AF062EC46F0FF0E3F
:1052600058EC2AF032EC46F0FF0E58EC2AF0B2EC83
:1052700045F0FF0E58EC2AF015EF2AF0FF0E58EC1F
:105280002AF0D2EC45F0FF0E58EC2AF092EC46F0F2
:10529000FF0E58EC2AF0C2EC45F0FF0E58EC2AF055
:1052A000C2EC45F0FF0E58EC2AF015EF2AF01DEC89
:1052B0002AF0460E26EC2AF0BB0E3FEC2AF04DA257
:1052C00094EF29F0FF0E58EC2AF002EC46F0FF0EA6
:1052D00058EC2AF052EC46F0FF0E58EC2AF0B2ECF3
:1052E00046F0FF0E58EC2AF0C2EC45F0FF0E58ECE9
:1052F0002AF092EC46F0FF0E58EC2AF032EC46F021
:10530000FF0E58EC2AF062EC46F0FF0E58EC2AF043
:10531000A2EC45F0FF0E58EC2AF022EC46F0FF0E0E
:1053200058EC2AF015EF2AF0FF0E58EC2AF0D2ECD8
:1053300045F0FF0E58EC2AF092EC46F0FF0E58ECC8
:105340002AF0C2EC45F0FF0E58EC2AF0C2EC45F012
:10535000FF0E58EC2AF022EC47F0000E58EC2AF031
:1053600022EC47F0000E58EC2AF022EC47F0000E39
:1053700058EC2AF022EC47F0000E58EC2AF022EC10
:1053800047F0000E58EC2AF015EF2AF01DEC2AF039
:10539000460E26EC2AF0BC0E3FEC2AF04DA4F4EFAA
:1053A00029F0FF0E58EC2AF082EC45F0FF0E58EC85
:1053B0002AF0C2EC46F0FF0E58EC2AF0B2EC46F0B0
:1053C000FF0E58EC2AF062EC46F0FF0E58EC2AF083
:1053D00022EC47F0000E58EC2AF022EC47F0000EC9
:1053E00058EC2AF015EF2AF0FF0E58EC2AF042ECA8
:1053F00046F0FF0E58EC2AF082EC45F0FF0E58EC18
:105400002AF052EC46F0FF0E58EC2AF0C2EC46F0BF
:10541000FF0E58EC2AF082EC45F0FF0E58EC2AF013
:1054200032EC46F0FF0E58EC2AF04CAEDBEC2DF0DF
:105430001BEF01F08C888B9E12008C988B8E1200D3
:105440008C888B8E12008C988B9E1200016E1FEC44
:105450002BF001508A6E8C9C8C9E000000008C8A80
:10546000000000000000000000000000000000003C
:105470008C9A000000000000000000001200026E84
:105480001FEC2BF002508A6E8C9C8C9E000000005A
:105490008C8A0000000000000000000000000000F6
:1054A00000008C9A000000000000000000001200C4
:1054B000006E1FEC2BF03FBE74EC2AF000508A6E99
:1054C0008C9C8C8E000000008C8A00000000000084
:1054D000000000000000000000008C9A00000000A6
:1054E0000000000000001200000E515CD8B499EFDB
:1054F0002AF0010E515CD8B4B2EF2AF0020E515CD2
:10550000D8B4C9EF2AF0030E515CD8B4DEEF2AF00C
:10551000040E515CD8B4F1EF2AF0050E515CD8B4FA
:1055200002EF2BF0060E515CD8B411EF2BF01EEFFA
:105530002BF050B0A7EF2AF0004200420042004298
:10554000004200420042010E00161EEF2BF0004602
:10555000004600460046004600460046800E001603
:105560001EEF2BF050B0BFEF2AF000420042004285
:10557000004200420042030E00161EEF2BF00046D0
:1055800000460046004600460046C00E00161EEFCC
:105590002BF050B0D5EF2AF000420042004200420A
:1055A0000042070E00161EEF2BF000460046004694
:1055B00000460046E00E00161EEF2BF050B0E9EF5B
:1055C0002AF000420042004200420F0E00161EEF79
:1055D0002BF00046004600460046F00E00161EEF77
:1055E0002BF050B0FBEF2AF00042004200421F0EA9
:1055F00000161EEF2BF0004600460046F80E00167F
:105600001EEF2BF050B00BEF2BF0004200423F0E8C
:1056100000161EEF2BF000460046FC0E00161EEF93
:105620002BF050B019EF2BF000427F0E00161EEF4A
:105630002BF00046FE0E00161EEF2BF012000F019D
:10564000FF0E936E00018C8C8C9E000000008C8AF3
:10565000000000000000000000000000000000004A
:105660008C9A000000000000000000000000000014
:10567000000081BE27EF2BF08C9C0F01000E936E73
:105680000001120020EC2AF0400E26EC2AF0B80EA1
:105690003FEC2AF0000E58EC2AF0012A800E015C43
:1056A000D8A44AEF2BF0022A40EC2AF0400E26EC58
:1056B0002AF0C00E025CD8A44AEF2BF012008B80B7
:1056C00000008B92DBEC35F08B82DBEC35F07CEC70
:1056D0002BF092EC2BF0A7EC2BF0BCEC2BF0D1ECE8
:1056E0002BF0E6EC2BF0FBEC2BF010EC2CF025EC87
:1056F0002CF03AEC2CF012008B9000004FEC2CF0C8
:105700008B9400008B8600008B960000000E386E94
:105710007AEC2CF011503C6E8FEC2CF08B948B9625
:105720008B8012008B904FEC2CF08B9400008B86BA
:1057300000008B960000010E386E7AEC2CF01250AF
:105740003C6E8FEC2CF08B948B968B8012008B90A0
:105750004FEC2CF08B9400008B8600008B960000A1
:10576000020E386E7AEC2CF013503C6E8FEC2CF05D
:105770008B948B968B8012008B904FEC2CF08B943B
:1057800000008B8600008B960000030E386E7AECCA
:105790002CF014503C6E8FEC2CF08B948B968B80FD
:1057A00012008B904FEC2CF08B9400008B86000045
:1057B0008B960000040E386E7AEC2CF015503C6E7F
:1057C0008FEC2CF08B948B968B8012008B904FEC8F
:1057D0002CF08B9400008B8600008B960000050E49
:1057E000386E7AEC2CF016503C6E8FEC2CF08B94CB
:1057F0008B968B8012008B904FEC2CF08B940000DA
:105800008B8600008B960000060E386E7AEC2CF02A
:1058100017503C6E8FEC2CF08B948B968B80120083
:105820008B904FEC2CF08B9400008B8600008B96B5
:105830000000070E386E7AEC2CF018503C6E8FEC9E
:105840002CF08B948B968B8012008B904FEC2CF06D
:105850008B9400008B8600008B960000080E386E3B
:105860007AEC2CF019503C6E8FEC2CF08B948B96CC
:105870008B8012008B904FEC2CF08B9400008B8669
:1058800000008B960000090E386E7AEC2CF01A504E
:105890003C6E8FEC2CF08B948B968B8012008B944B
:1058A00000008B8600008B9600008B9400008B8696
:1058B00000008B9600008B8400008B8600008B9686
:1058C00000008B9400008B8600008B9600008B9468
:1058D00000008B8600008B9600008B9400008B8666
:1058E00000008B9600008B9400008B8600008B9646
:1058F0000000120038BE80EF2CF08B9482EF2CF069
:105900008B8400008B8600008B960000392A384675
:10591000080E395CD8A47AEF2CF0396A12003CBE2C
:1059200095EF2CF08B9497EF2CF08B8400008B86F6
:1059300000008B9600003A2A3C46080E3A5CD8A438
:105940008FEF2CF03A6A12008B904FEC2CF08B9476
:1059500000008B8600008B9600000A0E386E7AECF1
:105960002CF08B800000000000008B904FEC2CF09E
:105970008B8400008B8600008B96000000000000E6
:105980000000C7EC2CF08B948B968B8012008B86DA
:1059900083A0CEEF2CF03B80CFEF2CF03B903A2A47
:1059A0008B96080E3A5CD8B4D9EF2CF03B46C7EF83
:1059B0002CF03A6A3D2A010E3D5CD8A4E4EF2CF0AD
:1059C0003B501B6EC7EF2CF0020E3D5CD8A4EDEFF0
:1059D0002CF03B501C6EC7EF2CF0030E3D5CD8A49E
:1059E000F6EF2CF03B501D6EC7EF2CF0040E3D5C23
:1059F000D8A4FFEF2CF03B501E6EC7EF2CF0050E25
:105A00003D5CD8A408EF2DF03B501F6EC7EF2CF083
:105A1000060E3D5CD8A411EF2DF03B50206EC7EF71
:105A20002CF0070E3D5CD8A41AEF2DF03B50216EF0
:105A3000C7EF2CF0080E3D5CD8A423EF2DF03B50AF
:105A4000226EC7EF2CF0090E3D5CD8A42CEF2DF090
:105A50003B50236EC7EF2CF00A0E3D5CD8A435EF07
:105A60002DF03B50246EC7EF2CF00B0E3D5CD8A4FC
:105A70003EEF2DF03B50256EC7EF2CF00C0E3D5C39
:105A8000D8A447EF2DF03B50266EC7EF2CF00D0E3B
:105A90003D5CD8A450EF2DF03B50276EC7EF2CF0A3
:105AA0000E0E3D5CD8A459EF2DF03B50286EC7EF89
:105AB0002CF00F0E3D5CD8A462EF2DF03B50296E08
:105AC000C7EF2CF0100E3D5CD8A46BEF2DF03B50CF
:105AD0002A6EC7EF2CF0110E3D5CD8A474EF2DF0A8
:105AE0003B502B6EC7EF2CF0120E3D5CD8A47DEF1F
:105AF0002DF03B502C6EC7EF2CF0130E3D5CD8A45C
:105B000086EF2DF03B502D6EC7EF2CF0140E3D5C50
:105B1000D8A48FEF2DF03B502E6EC7EF2CF0150E52
:105B20003D5CD8A498EF2DF03B502F6EC7EF2CF0C2
:105B3000160E3D5CD8A4A1EF2DF03B50306EC7EFA0
:105B40002CF0170E3D5CD8A4AAEF2DF03B50316E1F
:105B5000C7EF2CF0180E3D5CD8A4B3EF2DF03B50EE
:105B6000326EC7EF2CF0190E3D5CD8A4BCEF2DF0BF
:105B70003B50336EC7EF2CF01A0E3D5CD8A4C5EF36
:105B80002DF03B50346EC7EF2CF01B0E3D5CD8A4BB
:105B9000CEEF2DF03B50356EC7EF2CF01C0E3D5C68
:105BA000D8A4D7EF2DF03B50366EC7EF2CF03B500A
:105BB000376E3D6A120080BAE8EF2DF03EBA12004F
:105BC00042EC2BF0416A466A476A486A3E8A1200F4
:105BD0003E9A1200000E405CD8A413EF2EF052EC57
:105BE00044F0000E58EC2AF0B2EC44F0000E58ECF1
:105BF0002AF022EC44F0000E58EC2AF022EC47F098
:105C0000000E58EC2AF022EC47F0000E58EC2AF077
:105C100022EC47F0000E58EC2AF022EC47F0000E80
:105C200058EC2AF01200010E405CD8A43CEF2EF094
:105C300032EC44F0000E58EC2AF0A2EC44F0000ED6
:105C400058EC2AF0D2EC44F0000E58EC2AF062EC4A
:105C500044F0000E58EC2AF022EC47F0000E58EC0D
:105C60002AF022EC47F0000E58EC2AF022EC47F024
:105C7000000E58EC2AF01200020E405CD8A465EF2A
:105C80002EF072EC44F0000E58EC2AF0B2EC44F026
:105C9000000E58EC2AF012EC45F0000E58EC2AF0F9
:105CA00022EC47F0000E58EC2AF022EC47F0000EF0
:105CB00058EC2AF022EC47F0000E58EC2AF022ECC7
:105CC00047F0000E58EC2AF01200030E405CD8A4F6
:105CD0008EEF2EF012EC44F0000E58EC2AF022EC7D
:105CE00047F0000E58EC2AF002EC45F0000E58EC9C
:105CF0002AF012EC45F0000E58EC2AF0F2EC43F0DA
:105D0000000E58EC2AF022EC47F0000E58EC2AF076
:105D100022EC47F0000E58EC2AF01200040E405C12
:105D2000D8A4B7EF2EF022EC45F0000E58EC2AF084
:105D300022EC47F0000E58EC2AF022EC44F0000E62
:105D400058EC2AF0F2EC43F0000E58EC2AF012EC7A
:105D500045F0000E58EC2AF0F2EC43F0000E58EC3F
:105D60002AF022EC47F0000E58EC2AF01200050E43
:105D7000405CD8A4E0EF2EF0F2EC44F0000E58ECBA
:105D80002AF022EC47F0000E58EC2AF032EC44F0F6
:105D9000000E58EC2AF0F2EC44F0000E58EC2AF019
:105DA000F2EC44F0000E58EC2AF022EC47F0000E22
:105DB00058EC2AF022EC47F0000E58EC2AF01200C2
:105DC000060E405CD8A409EF2FF0B2EC44F0000EB0
:105DD00058EC2AF032EC45F0000E58EC2AF022EC98
:105DE00047F0000E58EC2AF032EC44F0000E58EC6C
:105DF0002AF0F2EC44F0000E58EC2AF0F2EC44F0F9
:105E0000000E58EC2AF022EC47F0000E58EC2AF075
:105E10001200070E405CD8A432EF2FF0F2EC44F0F1
:105E2000000E58EC2AF012EC44F0000E58EC2AF068
:105E300002EC44F0000E58EC2AF092EC44F0000E14
:105E400058EC2AF022EC47F0000E58EC2AF022EC35
:105E500047F0000E58EC2AF022EC47F0000E58EC08
:105E60002AF01200080E405CD8A45BEF2FF0A2ECE1
:105E700041F0000E58EC2AF072EC41F0000E58ECA4
:105E80002AF082EC44F0000E58EC2AF062EC44F068
:105E9000000E58EC2AF072EC45F0000E58EC2AF097
:105EA00022EC47F0000E58EC2AF022EC47F0000EEE
:105EB00058EC2AF01200090E405CD8A484EF2FF0B1
:105EC000F2EC43F0000E58EC2AF022EC45F0000E04
:105ED00058EC2AF022EC44F0000E58EC2AF072EC58
:105EE00044F0000E58EC2AF0C2EC44F0000E58ECDE
:105EF0002AF022EC47F0000E58EC2AF022EC47F092
:105F0000000E58EC2AF012000A0E405CD8A4ADEF47
:105F10002FF032EC45F0000E58EC2AF092EC44F0F1
:105F2000000E58EC2AF0F2EC44F0000E58EC2AF087
:105F300012EC44F0000E58EC2AF082EC44F0000E13
:105F400058EC2AF022EC47F0000E58EC2AF022EC34
:105F500047F0000E58EC2AF012000B0E405CD8A45B
:105F60008FEF30F012EC45F0000E58EC2AF052ECB6
:105F700045F0000E58EC2AF022EC47F0000E58ECE9
:105F80002AF01550070B406E000E405CD8A4DEEFDF
:105F90002FF0F2EC44F0000E58EC2AF052EC45F0F1
:105FA000000E58EC2AF0D2EC44F0000E58EC2AF027
:105FB00012EC41F0000E58EC2AF01200010E405C89
:105FC000D8A4F8EF2FF0F2EC44F0000E58EC2AF0D1
:105FD00052EC45F0000E58EC2AF0D2EC44F0000EE2
:105FE00058EC2AF022EC41F0000E58EC2AF0120096
:105FF000020E405CD8A412EF30F0F2EC44F0000E38
:1060000058EC2AF052EC45F0000E58EC2AF0D2EC95
:1060100044F0000E58EC2AF032EC41F0000E58EC3F
:106020002AF01200030E405CD8A42CEF30F022ECD2
:1060300045F0000E58EC2AF002EC45F0000E58EC4A
:106040002AF002EC44F0000E58EC2AF022EC47F063
:10605000000E58EC2AF01200040E405CD8A446EF63
:1060600030F0F2EC44F0000E58EC2AF052EC45F01F
:10607000000E58EC2AF0D2EC44F0000E58EC2AF056
:1060800052EC41F0000E58EC2AF01200050E405C74
:10609000D8A460EF30F0F2EC44F0000E58EC2AF097
:1060A00052EC45F0000E58EC2AF0D2EC44F0000E11
:1060B00058EC2AF062EC41F0000E58EC2AF0120085
:1060C000060E405CD8A47AEF30F0F2EC44F0000EFB
:1060D00058EC2AF052EC45F0000E58EC2AF0D2ECC5
:1060E00044F0000E58EC2AF072EC41F0000E58EC2F
:1060F0002AF01200F2EC44F0000E58EC2AF052ECB8
:1061000045F0000E58EC2AF0D2EC44F0000E58ECAA
:106110002AF082EC41F0000E58EC2AF012000C0E2E
:10612000405CD8A4B8EF30F032EC45F0000E58ECEB
:106130002AF022EC44F0000E58EC2AF022EC44F055
:10614000000E58EC2AF022EC47F0000E58EC2AF032
:1061500022EC47F0000E58EC2AF022EC47F0000E3B
:1061600058EC2AF022EC47F0000E58EC2AF012000E
:106170000D0E405CD8A4E1EF30F062EC44F0000E6C
:1061800058EC2AF0F2EC44F0000E58EC2AF0A2ECA5
:1061900044F0000E58EC2AF012EC44F0000E58ECDB
:1061A0002AF082EC44F0000E58EC2AF022EC47F082
:1061B000000E58EC2AF022EC47F0000E58EC2AF0C2
:1061C0001200F2EC44F0000E58EC2AF032EC44F0ED
:1061D000000E58EC2AF002EC45F0000E58EC2AF0C4
:1061E00032EC44F0000E58EC2AF0F2EC44F0000ED1
:1061F00058EC2AF032EC45F0000E58EC2AF032EC64
:1062000044F0000E58EC2AF0120080B018EF31F084
:106210003EB019EF31F0000E495CD8A414EF31F014
:10622000080E496E15EF31F049063E8019EF31F046
:106230003E9084B62CEF31F03EBC2DEF31F0080ECD
:10624000495CD8A428EF31F0000E496E29EF31F0F7
:10625000492A3E8C2DEF31F03E9C120080B041EF78
:1062600031F03EB042EF31F0010E495CD8A43DEF71
:1062700031F0080E496E3EEF31F049063E8042EFA4
:1062800031F03E9084B655EF31F03EBC56EF31F020
:10629000080E495CD8A451EF31F0010E496E52EF5F
:1062A00031F0492A3E8C56EF31F03E9C1200080E28
:1062B000495CD8B43BEF33F03FB493EF31F080B892
:1062C00069EF31F03EB826EF32F03F843E8893EF1D
:1062D00031F03E981AEC2AF04D0E26EC2AF0BE0E54
:1062E0003FEC2AF0000E58EC2AF022EC47F0000EAA
:1062F00058EC2AF022EC47F022EC47F0000E58EC64
:106300002AF022EC47F0000E58EC2AF022EC47F07D
:10631000000E58EC2AF022EC47F0000E58EC2AF060
:106320004A50406E12001AEC2AF04D0E26EC2AF06C
:10633000BE0E3FEC2AF0000E495CD8B4C0EF31F03D
:10634000010E495CD8B4C5EF31F0020E495CD8B4F7
:10635000CAEF31F0030E495CD8B4CFEF31F0040E30
:10636000495CD8B4D4EF31F0050E495CD8B4D9EF0C
:1063700031F0060E495CD8B4DEEF31F0E3EF31F0D6
:106380004BAEE8EF31F008EF32F04BACE8EF31F014
:1063900008EF32F04BAAE8EF31F008EF32F04BA8EB
:1063A000E8EF31F008EF32F04BA6E8EF31F008EFFC
:1063B00032F04BA4E8EF31F008EF32F04BA2E8EFF7
:1063C00031F008EF32F04BA0E8EF31F008EF32F097
:1063D000000E58EC2AF022EC41F0000E58EC2AF0A6
:1063E00022EC47F0C2EC44F0000E58EC2AF0F2EC3C
:1063F00044F0000E58EC2AF022EC47F0FF0E58EC67
:106400002AF0B2EC41F0FF0E58EC2AF026EF32F001
:10641000FF0E58EC2AF0C2EC41F0FF0E58EC2AF0C7
:1064200022EC47F0C2EC44F0000E58EC2AF0F2ECFB
:1064300044F0000E58EC2AF022EC47F0000E58EC25
:106440002AF012EC41F0000E58EC2AF04A50406E4F
:106450003FA4120080BA35EF32F03EBA36EF32F088
:106460003F944A50406E3E8A12003E9A80B8AFEF89
:1064700032F03EB8B0EF32F0000E495CD8B461EFB4
:1064800032F0010E495CD8B46AEF32F0020E495C7A
:10649000D8B473EF32F0030E495CD8B47CEF32F01D
:1064A000040E495CD8B485EF32F0050E495CD8B4CF
:1064B0008EEF32F0060E495CD8B497EF32F0A0EFC1
:1064C00032F04BAE67EF32F04A8EA9EF32F04A9EBF
:1064D000A9EF32F04BAC70EF32F04A8CA9EF32F0FA
:1064E0004A9CA9EF32F04BAA79EF32F04A8AA9EF21
:1064F00032F04A9AA9EF32F04BA882EF32F04A8884
:10650000A9EF32F04A98A9EF32F04BA68BEF32F0A8
:106510004A86A9EF32F04A96A9EF32F04BA494EFE5
:1065200032F04A84A9EF32F04A94A9EF32F04BA23C
:106530009DEF32F04A82A9EF32F04A92A9EF32F091
:106540004BA0A6EF32F04A80A9EF32F04A90A9EFB3
:1065500032F03F944A50406E3E88B0EF32F03E98A1
:1065600080B0F4EF32F03EB0F5EF32F0000E495C4F
:10657000D8B4DBEF32F0010E495CD8B4DEEF32F074
:10658000020E495CD8B4E1EF32F0030E495CD8B496
:10659000E4EF32F0040E495CD8B4E7EF32F0050EB8
:1065A000495CD8B4EAEF32F0060E495CD8B4EDEF9E
:1065B00032F0F0EF32F04B7EF1EF32F04B7CF1EF46
:1065C00032F04B7AF1EF32F04B78F1EF32F04B765C
:1065D000F1EF32F04B74F1EF32F04B72F1EF32F039
:1065E0004B703E80F5EF32F03E9084B639EF33F0D9
:1065F0003EBC3AEF33F0000E495CD8B420EF33F0E4
:10660000010E495CD8B423EF33F0020E495CD8B4D4
:1066100026EF33F0030E495CD8B429EF33F0040EB3
:10662000495CD8B42CEF33F0050E495CD8B42FEF99
:1066300033F0060E495CD8B432EF33F035EF33F067
:106640004B7E36EF33F04B7C36EF33F04B7A36EF40
:1066500033F04B7836EF33F04B7636EF33F04B7444
:1066600036EF33F04B7236EF33F04B703E8C3AEF2F
:1066700033F03E9C120080B8ACEF33F03EB8ADEF83
:1066800033F0000E465CD8B474EF33F0010E465C74
:10669000D8B478EF33F0020E465CD8B47CEF33F018
:1066A000030E465CD8B480EF33F0040E465CD8B4D9
:1066B00084EF33F0050E465CD8B488EF33F0060E55
:1066C000465CD8B48CEF33F0070E465CD8B490EF3C
:1066D00033F0080E465CD8B494EF33F0090E465CF4
:1066E000D8B498EF33F012004A50116E9AEF33F09D
:1066F0004A50126E9AEF33F04A50136E9AEF33F00D
:106700004A50146E9AEF33F04A50156E9AEF33F0F8
:106710004A50166E9AEF33F04A50176E9AEF33F0E4
:106720004A50186E9AEF33F04A50196E9AEF33F0D0
:106730004A501A6E5FEC2BF04A50406E3E88000EB5
:10674000465CD8B4A8EF33F0070E496EADEF33F0D6
:10675000050E496EADEF33F03E9812001AEC2AF0A8
:10676000670E26EC2AF0BC0E3FEC2AF03FBCCDEFC2
:1067700033F0000E58EC2AF062EC45F0000E58ECB5
:106780002AF032EC44F0000E58EC2AF002EC45F00E
:10679000000E58EC2AF0DFEF33F0FF0E58EC2AF031
:1067A00002EC47F0FF0E58EC2AF0C2EC45F0FF0E69
:1067B00058EC2AF0A2EC46F0FF0E58EC2AF01DEC43
:1067C0002AF0440E26EC2AF0BC0E3FEC2AF03FBC27
:1067D000FEEF33F0FF0E58EC2AF052EC46F0FF0EBD
:1067E00058EC2AF032EC47F0FF0E58EC2AF062EC3D
:1067F00046F0FF0E58EC2AF010EF34F0000E58EC83
:106800002AF0B2EC44F0000E58EC2AF022EC47F0EB
:10681000000E58EC2AF0C2EC44F0000E58EC2AF0BE
:1068200080B020EF34F03EB021EF34F03FBC1CEFDD
:1068300034F03F8C1DEF34F03F9C3E8021EF34F06C
:106840003E9084B631EF34F03EBC32EF34F03FBCC2
:106850002DEF34F03F8C2EEF34F03F9C3E8C32EF26
:1068600034F03E9C120080B8A7EF34F03EB8A8EF99
:1068700034F03FACA1EF34F042EC2BF0000E475C5B
:10688000D8B477EF34F0010E475CD8B47BEF34F026
:10689000020E475CD8B47FEF34F0030E475CD8B4E7
:1068A00083EF34F0040E475CD8B487EF34F0050E64
:1068B000475CD8B48BEF34F0060E475CD8B48FEF4A
:1068C00034F0070E475CD8B493EF34F0080E475C01
:1068D000D8B497EF34F0090E475CD8B49BEF34F08E
:1068E0000A0E475CD8B49FEF34F0A1EF34F05AECB5
:1068F00047F0A1EF34F06DEC47F0A1EF34F080ECFD
:1069000047F0A1EF34F093EC47F0A1EF34F0A6ECA0
:1069100047F0A1EF34F0B9EC47F0A1EF34F0CCEC44
:1069200047F0A1EF34F0DFEC47F0A1EF34F0F2ECE8
:1069300047F0A1EF34F005EC48F0A1EF34F018EC8B
:1069400048F0446A476A3F9C3E881BEF01F03E983E
:10695000120083A2C9EF34F03FB812004CB2BBEF73
:1069600034F01550380B406E180E406E1550C70BA2
:10697000156EC3EF34F015503F0B406E1B0E406E8A
:106980001550C00B156E405015125FEC2BF03F8870
:1069900012003F9812001550380B406E40424042A2
:1069A00040424050070B406E1550F80B156E40509A
:1069B00015121200106E000E105CD8A4F8EF34F01F
:1069C00005B8E9EF34F005BAEDEF34F072EC40F0C1
:1069D000120022EC47F0058C120005BCF4EF34F0F5
:1069E000059C72EC40F01200059C22EC47F012006E
:1069F000010E105CD8A400EF35F082EC40F01200DC
:106A0000020E105CD8A408EF35F092EC40F01200B2
:106A1000030E105CD8A410EF35F0A2EC40F0120089
:106A2000040E105CD8A418EF35F0B2EC40F0120060
:106A3000050E105CD8A420EF35F0C2EC40F0120037
:106A4000060E105CD8A428EF35F0D2EC40F012000E
:106A5000070E105CD8A430EF35F0E2EC40F01200E5
:106A6000080E105CD8A438EF35F0F2EC40F01200BC
:106A700002EC41F01200106E000E105CD8A444EF3E
:106A800035F012EC41F01200010E105CD8A44CEF6E
:106A900035F022EC41F01200020E105CD8A454EF45
:106AA00035F032EC41F01200030E105CD8A45CEF1C
:106AB00035F042EC41F01200040E105CD8A464EFF3
:106AC00035F052EC41F01200050E105CD8A46CEFCA
:106AD00035F062EC41F01200060E105CD8A474EFA1
:106AE00035F072EC41F01200070E105CD8A47CEF78
:106AF00035F082EC41F01200080E105CD8A484EF4F
:106B000035F092EC41F01200A2EC41F01200106E50
:106B1000000E105CD8A490EF35F0B2EC41F01200FA
:106B2000010E105CD8A498EF35F0C2EC41F01200D1
:106B3000020E105CD8A4A0EF35F0D2EC41F01200A8
:106B4000030E105CD8A4A8EF35F0E2EC41F012007F
:106B5000040E105CD8A4B0EF35F0F2EC41F0120056
:106B6000050E105CD8A4B8EF35F002EC42F012002C
:106B7000060E105CD8A4C0EF35F012EC42F0120003
:106B8000070E105CD8A4C8EF35F022EC42F01200DA
:106B9000080E105CD8A4D0EF35F032EC42F01200B1
:106BA00042EC42F01200062A0A0E065CD8A4D3EF8B
:106BB00035F0066A1200062AFF0E065CD8A4DBEF49
:106BC00035F0066A072A640E075CD8A4DBEF35F0BF
:106BD000066A076A1200062AFF0E065CD8A4EBEFCD
:106BE00035F0066A072AFF0E075CD8A4EBEF35F0F4
:106BF000066A076A12001AEC2AF0400E26EC2AF008
:106C0000BF0E3FEC2AF022EC44F0000E58EC2AF0C4
:106C1000F2EC43F0000E58EC2AF072EC44F0000E57
:106C200058EC2AF092EC41F0000E58EC2AF052ECAD
:106C300041F0000E58EC2AF022EC41F0000E58EC26
:106C40002AF072EC41F022EC47F0F2EC44F0000E36
:106C500058EC2AF032EC44F0000E58EC2AF032ECFA
:106C600045F01DEC2AF0400E26EC2AF0BF0E3FEC5A
:106C70002AF0400E58EC2AF0000E58EC2AF022ECD4
:106C800041F0000E58EC2AF0400E58EC2AF0000EAD
:106C900058EC2AF012EC41F0000E58EC2AF0400EAD
:106CA000036E7F0E046E1AEC2AF0035026EC2AF0D5
:106CB000BC0E3FEC2AF0010E58EC2AF01DEC2AF035
:106CC000045026EC2AF0BC0E3FEC2AF0010E58ECE2
:106CD0002AF0032A0406DBEC35F0800E035CD8A40E
:106CE00053EF36F0EBEC35F0EBEC35F0EBEC35F048
:106CF000EBEC35F0EBEC35F0400E036E7F0E046EDE
:106D00001AEC2AF0035026EC2AF0BC0E3FEC2AF0D5
:106D1000000E58EC2AF01DEC2AF0045026EC2AF064
:106D2000BC0E3FEC2AF0000E58EC2AF0032A0406B1
:106D3000DBEC35F0800E035CD8A480EF36F03F8E9C
:106D4000EBEC35F0EBEC35F0EBEC35F0EBEC35F053
:106D500050801AEC2AF04A0E26EC2AF0BB0E3FECCB
:106D60002AF0A2EC42F0000E58EC2AF0100E58EC7B
:106D70002AF0100E58EC2AF0100E58EC2AF0100EE3
:106D800058EC2AF0100E58EC2AF0000E58EC2AF0BD
:106D900022EC43F0000E58EC2AF022EC47F0000EF3
:106DA00058EC2AF092EC42F0000E58EC2AF022EC5B
:106DB00043F0000E58EC2AF0B2EC42F0000E58EC12
:106DC0002AF0D2EC42F0000E58EC2AF022EC43F00C
:106DD000000E58EC2AF01DEC2AF0400E26EC2AF0AA
:106DE000BB0E3FEC2AF092EC42F0000E58EC2AF079
:106DF00092EC42F0000E58EC2AF062EC43F0000EE8
:106E000058EC2AF0D2EC42F0000E58EC2AF022ECBA
:106E100043F0000E58EC2AF0B2EC42F0000E58ECB1
:106E20002AF050901AEC2AF0560E26EC2AF0BC0EEE
:106E30003FEC2AF052EC42F0000E58EC2AF092ECB3
:106E400043F0000E58EC2AF082EC42F0000E58ECB1
:106E50002AF0D2EC42F0000E58EC2AF032EC43F06B
:106E6000000E58EC2AF022EC47F0000E58EC2AF005
:106E700002EC43F0000E58EC2AF01DEC2AF0400E14
:106E800026EC2AF0BC0E3FEC2AF052EC42F0000E49
:106E900058EC2AF062EC42F0000E58EC2AF032EC8A
:106EA00043F0000E58EC2AF062EC43F0000E58EC70
:106EB0002AF052EC42F0000E58EC2AF082EC43F03B
:106EC000000E58EC2AF032EC43F0000E58EC2AF099
:106ED00062EC43F0000E58EC2AF0D2EC43F0000EC6
:106EE00058EC2AF0512A080E515CD8A4A0EF36F0D5
:106EF0003F9E516AEBEC35F0EBEC35F0EBEC35F006
:106F0000EBEC35F0EBEC35F0EBEC35F0EBEC35F091
:106F1000EBEC35F0EBEC35F0EBEC35F0EBEC35F081
:106F2000EBEC35F0EBEC35F0EBEC35F0EBEC35F071
:106F3000EBEC35F0EBEC35F0EBEC35F0EBEC35F061
:106F4000EBEC35F0EBEC35F0EBEC35F0EBEC35F051
:106F5000EBEC35F0EBEC35F0EBEC35F0EBEC35F041
:106F6000EBEC35F0EBEC35F0EBEC35F0EBEC35F031
:106F7000EBEC35F0EBEC35F0EBEC35F0EBEC35F021
:106F8000EBEC35F0EBEC35F0EBEC35F0EBEC35F011
:106F9000EBEC35F0EBEC35F0EBEC35F0EBEC35F001
:106FA000EBEC35F0EBEC35F0EBEC35F0EBEC35F0F1
:106FB000EBEC35F0EBEC35F0EBEC35F0EBEC35F0E1
:106FC000EBEC35F0EBEC35F0EBEC35F0EBEC35F0D1
:106FD000EBEC35F0EBEC35F0EBEC35F0EBEC35F0C1
:106FE000EBEC35F0EBEC35F0EBEC35F0EBEC35F0B1
:106FF000EBEC35F0EBEC35F0EBEC35F0EBEC35F0A1
:10700000EBEC35F0EBEC35F0EBEC35F0EBEC35F090
:10701000EBEC35F0EBEC35F0EBEC35F042EC2BF033
:10702000EBEC35F0EBEC35F0EBEC35F0EBEC35F070
:107030001200096E640E095ED8A022EF38F00A2A09
:107040001AEF38F0640E09260A0E095ED8A02CEF5C
:1070500038F00B2A24EF38F00A0E0926010E095EDB
:10706000D8A036EF38F00C2A2EEF38F012000D6E53
:10707000100E0D5ED8A040EF38F00B2A38EF38F034
:10708000100E0D26010E0D5ED8A04AEF38F00C2A26
:1070900042EF38F0120005880A50DAEC34F0000EA6
:1070A00058EC2AF00598058A0B50DAEC34F0000E03
:1070B00058EC2AF0059A0C50DAEC34F0000E58EC3B
:1070C0002AF00A6A0B6A0C6A12000A503BEC35F08F
:1070D000000E58EC2AF00B503BEC35F0000E58EC4B
:1070E0002AF00C503BEC35F0000E58EC2AF00A6AFE
:1070F0000B6A0C6A12000A5087EC35F0FF0E58EC50
:107100002AF00B5087EC35F0FF0E58EC2AF00C50AB
:1071100087EC35F0FF0E58EC2AF00A6A0B6A0C6A0D
:107120001200406E452A090E455CD8B4A7EF38F02E
:1071300040BE9FEF38F012EC41F0A1EF38F022ECA6
:1071400041F0000E58EC2AF0404692EF38F0456AC4
:107150001200406E080E455CD8B4E6EF38F040BE31
:10716000CBEF38F04550495CD8B4C1EF38F0000E91
:1071700058EC2AF012EC41F0000E58EC2AF0E2EF45
:1071800038F0FF0E58EC2AF0B2EC41F0FF0E58EC4C
:107190002AF0E2EF38F04550495CD8B4DAEF38F025
:1071A000000E58EC2AF022EC41F0000E58EC2AF0C8
:1071B000E2EF38F0FF0E58EC2AF0C2EC41F0FF0E7F
:1071C00058EC2AF0452A4046AAEF38F0456A1200EA
:1071D0007D0E4F5CD8B4EFEF38F04F2A12003F8A93
:1071E0004F6A12001DEC2AF0530E26EC2AF0BE0E58
:1071F0003FEC2AF0080E495CD8A44AEF39F0FF0EA4
:1072000058EC2AF0A2EC46F0FF0E58EC2AF0C2EC43
:1072100045F0FF0E58EC2AF0B2EC46F0FF0E58ECA9
:107220002AF01AEC2AF0460E26EC2AF0BC0E3FECAF
:107230002AF0000E58EC2AF022EC47F0000E58EC31
:107240002AF022EC47F0000E58EC2AF022EC47F02E
:10725000000E58EC2AF022EC47F0000E58EC2AF011
:1072600022EC47F0000E58EC2AF022EC47F0000E1A
:1072700058EC2AF022EC47F0000E58EC2AF022ECF1
:1072800047F0000E58EC2AF022EC47F0000E58ECC4
:107290002AF01200000E58EC2AF002EC45F0000E25
:1072A00058EC2AF032EC44F0000E58EC2AF012ECC4
:1072B00045F0000E58EC2AF012001DEC2AF0400EAA
:1072C00026EC2AF0BB0E3FEC2AF01200000E58EC20
:1072D0002AF0B2EC44F0000E58EC2AF0C2EC44F074
:1072E000000E58EC2AF022EC47F0000E58EC2AF081
:1072F000E8EC3AF022EC47F0000E58EC2AF022ECD1
:1073000047F022EC47F043EC3BF01200FF0E58EC44
:107310002AF082EC46F0FF0E58EC2AF0A2EC45F081
:10732000FF0E58EC2AF092EC46F0FF0E58EC2AF0D3
:10733000A2EC45F0FF0E58EC2AF032EC47F0FF0EBD
:1073400058EC2AF002EC3BF043EC3BF01200FF0E4D
:1073500058EC2AF0A2EC45F0FF0E58EC2AF0A2EC13
:1073600045F0FF0E58EC2AF092EC46F0FF0E58EC78
:107370002AF0A2EC45F0FF0E58EC2AF032EC47F070
:10738000FF0E58EC2AF002EC3BF043EC3BF012000D
:10739000FF0E58EC2AF0C2EC46F0FF0E58EC2AF033
:1073A00052EC46F0FF0E58EC2AF032EC46F0FF0E9D
:1073B00058EC2AF062EC46F0FF0E58EC2AF0A2ECF2
:1073C00045F0FF0E58EC2AF022EC46F0FF0E58EC88
:1073D0002AF022EC47F0000E58EC2AF022EC47F09D
:1073E000000E58EC2AF022EC47F0000E58EC2AF080
:1073F00022EC47F0000E58EC2AF043EC3BF0120070
:10740000FF0E58EC2AF0D2EC46F0FF0E58EC2AF0B2
:1074100082EC45F0FF0E58EC2AF032EC46F0FF0EFD
:1074200058EC2AF002EC46F0FF0E58EC2AF0B2ECD1
:1074300045F0FF0E58EC2AF002EC46F0FF0E58EC37
:107440002AF0B2EC46F0FF0E58EC2AF002EC47F0BE
:10745000FF0E58EC2AF032EC47F0C2EC45F0FF0E7C
:1074600058EC2AF0810E58EC2AF0ED0E58EC2AF078
:10747000ED0E58EC2AF0ED0E58EC2AF05DEC39F0E8
:10748000930E58EC2AF0FF0E58EC2AF00CEC3BF06F
:1074900022EC47F0000E58EC2AF01200FF0E58ECD8
:1074A0002AF092EC45F0FF0E58EC2AF002EC46F080
:1074B000FF0E58EC2AF032EC47F0FF0E58EC2AF0A1
:1074C00072EC46F0FF0E58EC2AF0F2EC45F0FF0E9D
:1074D00058EC2AF082EC45F0FF0E58EC2AF0A2ECB2
:1074E00046F0FF0E58EC2AF0C2EC45F0FF0E58ECC7
:1074F0002AF032EC47F0C2EC45F0FF0E58EC2AF0CF
:10750000810E58EC2AF0ED0E58EC2AF0ED0E58ECF6
:107510002AF0ED0E58EC2AF05DEC39F0930E58ECA1
:107520002AF0FF0E58EC2AF00CEC3BF022EC47F06E
:10753000000E58EC2AF01200FF0E58EC2AF072EC04
:1075400046F0FF0E58EC2AF082EC45F0FF0E58ECA6
:107550002AF092EC46F0FF0E58EC2AF002EC46F0CE
:10756000FF0E58EC2AF0B2EC46F0FF0E58EC2AF071
:1075700002EC47F0FF0E58EC2AF032EC47F0C2EC78
:1075800045F0FF0E58EC2AF092EC46F0FF0E58EC56
:107590002AF092EC46F0FF0E58EC2AF0C30E58EC9D
:1075A0002AF0BD0E58EC2AF0BD0E58EC2AF0BD0EA4
:1075B00058EC2AF05DEC39F0C30E58EC2AF0FF0EBF
:1075C00058EC2AF016EC3BF0000E58EC2AF01200B2
:1075D00032EC44F0000E58EC2AF0F2EC44F0000ECD
:1075E00058EC2AF0F2EC44F0000E58EC2AF0C2EC11
:1075F00044F0000E58EC2AF0F2EC44F0000E58EC87
:107600002AF01200C2EC45F0FF0E58EC2AF092EC82
:1076100046F0FF0E58EC2AF092EC46F0FF0E58ECC4
:107620002AF062EC46F0FF0E58EC2AF092EC46F09D
:10763000FF0E58EC2AF0120002EC3BF032EC47F05F
:10764000FF0E58EC2AF0A2EC45F0FF0E58EC2AF0A1
:1076500062EC46F0FF0E58EC2AF0B2EC45F0FF0E5B
:1076600058EC2AF0C2EC45F0FF0E58EC2AF0FF0E61
:1076700058EC2AF0FF0E58EC2AF0FF0E58EC2AF0D6
:107680005DEC39F012005DEC39F022EC47F0000EB1
:1076900058EC2AF022EC47F0000E58EC2AF022ECCD
:1076A00047F0000E58EC2AF022EC47F0000E58ECA0
:1076B0002AF022EC47F0000E58EC2AF0120012ECEF
:1076C00044F0000E58EC2AF0C2EC44F0000E58ECE6
:1076D0002AF0B2EC44F0000E58EC2AF012EC45F01F
:1076E000000E58EC2AF0F2EC44F0000E58EC2AF0B0
:1076F000C2EC44F0000E58EC2AF092EC44F0000E7C
:1077000058EC2AF022EC47F012EC41F0000E58EC55
:107710002AF022EC47F01DEC2AF0400E26EC2AF06D
:10772000B90E3FEC2AF0FF0E58EC2AF0810E58EC0F
:107730002AF0810E58EC2AF0000E58EC2AF012ECD8
:1077400041F0000E58EC2AF012EC41F0000E58EC1B
:107750002AF062EC44F0000E58EC2AF0810E58EC4E
:107760002AF0810E58EC2AF0FF0E58EC2AF0120095
:1077700012EC44F0000E58EC2AF0C2EC44F0000E7B
:1077800058EC2AF0B2EC44F0000E58EC2AF012EC5F
:1077900045F0000E58EC2AF0F2EC44F0000E58ECE4
:1077A0002AF0C2EC44F0000E58EC2AF092EC44F0BF
:1077B000000E58EC2AF022EC47F022EC41F0000ECB
:1077C00058EC2AF022EC47F01DEC2AF0400E26EC93
:1077D0002AF0B90E3FEC2AF0FF0E58EC2AF0810E89
:1077E00058EC2AF0810E58EC2AF0000E58EC2AF0E2
:1077F00012EC41F0000E58EC2AF022EC41F0000EA1
:1078000058EC2AF062EC44F0000E58EC2AF0810E9D
:1078100058EC2AF0810E58EC2AF0FF0E58EC2AF0B2
:10782000120012EC44F0000E58EC2AF0C2EC44F0C6
:10783000000E58EC2AF0B2EC44F0000E58EC2AF09E
:1078400012EC45F0000E58EC2AF0F2EC44F0000E79
:1078500058EC2AF0C2EC44F0000E58EC2AF092ECFE
:1078600044F0000E58EC2AF022EC47F032EC41F0E4
:10787000000E58EC2AF022EC47F01DEC2AF0400EE6
:1078800026EC2AF0B90E3FEC2AF0FF0E58EC2AF055
:10789000810E58EC2AF0810E58EC2AF0000E58ECBC
:1078A0002AF012EC41F0000E58EC2AF032EC41F0D4
:1078B000000E58EC2AF062EC44F0000E58EC2AF06E
:1078C000810E58EC2AF0810E58EC2AF0FF0E58EC8D
:1078D0002AF0120012EC44F0000E58EC2AF0C2EC30
:1078E00044F0000E58EC2AF0B2EC44F0000E58ECD4
:1078F0002AF012EC45F0000E58EC2AF0F2EC44F0BD
:10790000000E58EC2AF0C2EC44F0000E58EC2AF0BD
:1079100092EC44F0000E58EC2AF022EC47F042ECD6
:1079200041F0000E58EC2AF022EC47F01DEC2AF052
:10793000400E26EC2AF0B90E3FEC2AF0FF0E58EC70
:107940002AF0810E58EC2AF0810E58EC2AF0000E35
:1079500058EC2AF012EC41F0000E58EC2AF042EC00
:1079600041F0000E58EC2AF062EC44F0000E58ECA6
:107970002AF0810E58EC2AF0810E58EC2AF0FF0E06
:1079800058EC2AF0120012EC44F0000E58EC2AF0E9
:10799000C2EC44F0000E58EC2AF0B2EC44F0000EB9
:1079A00058EC2AF012EC45F0000E58EC2AF0F2ECFC
:1079B00044F0000E58EC2AF0C2EC44F0000E58ECF3
:1079C0002AF092EC44F0000E58EC2AF022EC47F03A
:1079D00052EC41F0000E58EC2AF022EC47F01DEC7E
:1079E0002AF0400E26EC2AF0B90E3FEC2AF0FF0EEA
:1079F00058EC2AF0810E58EC2AF0810E58EC2AF04F
:107A0000000E58EC2AF012EC41F0000E58EC2AF06F
:107A100052EC41F0000E58EC2AF062EC44F0000EFB
:107A200058EC2AF0810E58EC2AF0810E58EC2AF01E
:107A3000FF0E58EC2AF0120002EC45F0000E58EC54
:107A40002AF032EC44F0000E58EC2AF0F2EC44F04C
:107A5000000E58EC2AF072EC44F0000E58EC2AF0BC
:107A6000F2EC43F0000E58EC2AF092EC44F0000ED9
:107A700058EC2AF022EC47F0F2EC43F0000E58EC00
:107A80002AF022EC45F0000E58EC2AF022EC44F0EB
:107A90001DEC2AF0400E26EC2AF0B90E3FEC2AF03D
:107AA000000E58EC2AF072EC44F0000E58EC2AF06C
:107AB000C2EC44F0000E58EC2AF01AEC2AF04C0EFE
:107AC00026EC2AF0BA0E3FEC2AF022EC44F0000E2D
:107AD00058EC2AF0F2EC43F0000E58EC2AF012ECCD
:107AE00045F0000E58EC2AF0F2EC43F0000E58EC92
:107AF0002AF022EC47F042EC44F0000E58EC2AF059
:107B0000C2EC44F0000E58EC2AF0F2EC44F0000E07
:107B100058EC2AF0A2EC44F01DEC2AF0400E26ECC2
:107B20002AF0BA0E3FEC2AF0000E58EC2AF0F2ECE4
:107B300043F0000E58EC2AF012EC45F022EC47F02E
:107B4000FF0E58EC2AF0810E58EC2AF0810E58EC0A
:107B50002AF0000E58EC2AF012EC41F0000E58EC1E
:107B60002AF062EC41F0000E58EC2AF062EC44F08E
:107B7000000E58EC2AF0810E58EC2AF0810E58ECD9
:107B80002AF0FF0E58EC2AF01200F2EC44F0000E3E
:107B900058EC2AF032EC44F0000E58EC2AF012ECCB
:107BA00044F0000E58EC2AF032EC44F0000E58EC91
:107BB0002AF072EC44F0000E58EC2AF032EC45F05A
:107BC000000E58EC2AF032EC44F0000E58EC2AF08B
:107BD000F2EC44F0000E58EC2AF022EC47F032ECC4
:107BE00044F01DEC2AF0400E26EC2AF0B90E3FECD2
:107BF0002AF0000E58EC2AF0F2EC44F0000E58EC9B
:107C00002AF0F2EC44F0000E58EC2AF0C2EC44F0FA
:107C1000000E58EC2AF0F2EC44F0000E58EC2AF07A
:107C200022EC47F0A2EC44F0000E58EC2AF0F2EC03
:107C300043F0000E58EC2AF002EC45F0000E58EC30
:107C40002AF082EC44F0000E58EC2AF01DEC2AF0E9
:107C5000640E26EC2AF0BA0E3FEC2AF0FF0E58EC28
:107C60002AF0810E58EC2AF0810E58EC2AF0000E12
:107C700058EC2AF012EC41F0000E58EC2AF072ECAD
:107C800041F0000E58EC2AF062EC44F0000E58EC83
:107C90002AF0810E58EC2AF0810E58EC2AF0FF0EE3
:107CA00058EC2AF0120072EC44F0000E58EC2AF066
:107CB000B2EC44F0000E58EC2AF012EC45F0000E45
:107CC00058EC2AF032EC44F0000E58EC2AF0F2ECBA
:107CD00044F0000E58EC2AF0F2EC44F0000E58ECA0
:107CE0002AF022EC45F0000E58EC2AF0D2EC44F0D9
:107CF000000E58EC2AF012EC45F022EC47F01DEC97
:107D00002AF0400E26EC2AF0B90E3FEC2AF0000EC5
:107D100058EC2AF0A2EC44F0000E58EC2AF0F2ECF9
:107D200043F0000E58EC2AF002EC45F0000E58EC3F
:107D30002AF082EC44F022EC47F0FF0E58EC2AF0D7
:107D4000810E58EC2AF0810E58EC2AF0000E58EC07
:107D50002AF012EC41F0000E58EC2AF082EC41F0CF
:107D6000000E58EC2AF062EC44F0000E58EC2AF0B9
:107D7000810E58EC2AF0810E58EC2AF0FF0E58ECD8
:107D80002AF0120072EC44F0000E58EC2AF0B2EC2B
:107D900044F0000E58EC2AF012EC45F0000E58ECBE
:107DA0002AF032EC44F0000E58EC2AF0F2EC44F0E9
:107DB000000E58EC2AF0F2EC44F0000E58EC2AF0D9
:107DC00022EC45F0000E58EC2AF0D2EC44F0000E04
:107DD00058EC2AF012EC45F022EC47F01DEC2AF0AA
:107DE000400E26EC2AF0B90E3FEC2AF0000E58ECBB
:107DF0002AF0A2EC44F0000E58EC2AF0C2EC44F059
:107E0000000E58EC2AF022EC44F0000E58EC2AF058
:107E100032EC44F0000E58EC2AF022EC47F0A2ECD1
:107E200044F0000E58EC2AF002EC45F0000E58EC3D
:107E30002AF002EC44F0000E58EC2AF01DEC2AF077
:107E4000640E26EC2AF0BA0E3FEC2AF0FF0E58EC36
:107E50002AF0810E58EC2AF0810E58EC2AF0000E20
:107E600058EC2AF012EC41F0000E58EC2AF092EC9B
:107E700041F0000E58EC2AF062EC44F0000E58EC91
:107E80002AF0810E58EC2AF0810E58EC2AF0FF0EF1
:107E900058EC2AF0120072EC44F0000E58EC2AF074
:107EA000B2EC44F0000E58EC2AF012EC45F0000E53
:107EB00058EC2AF032EC44F0000E58EC2AF0F2ECC8
:107EC00044F0000E58EC2AF0F2EC44F0000E58ECAE
:107ED0002AF022EC45F0000E58EC2AF0D2EC44F0E7
:107EE000000E58EC2AF012EC45F022EC47F01DECA5
:107EF0002AF0400E26EC2AF0B90E3FEC2AF0000ED4
:107F000058EC2AF0A2EC44F0000E58EC2AF0C2EC37
:107F100044F0000E58EC2AF022EC44F0000E58EC2D
:107F20002AF032EC44F0000E58EC2AF022EC47F034
:107F300092EC44F0000E58EC2AF002EC45F0000EF2
:107F400058EC2AF002EC44F0000E58EC2AF01DEC3C
:107F50002AF0640E26EC2AF0BA0E3FEC2AF0FF0E4F
:107F600058EC2AF0810E58EC2AF0810E58EC2AF0D9
:107F7000000E58EC2AF012EC41F0000E58EC2AF0FA
:107F8000A2EC41F0000E58EC2AF062EC44F0000E36
:107F900058EC2AF0810E58EC2AF0810E58EC2AF0A9
:107FA000FF0E58EC2AF01200FF0E58EC2AF072EC8B
:107FB00046F0FF0E58EC2AF0A2EC45F0FF0E58EC0C
:107FC0002AF0A2EC45F0FF0E58EC2AF0F2EC45F056
:107FD000FF0E58EC2AF01200FF0E58EC2AF062EC6B
:107FE00046F0FF0E58EC2AF0A2EC46F0FF0E58ECDB
:107FF0002AF032EC46F0FF0E58EC2AF002EC46F084
:10800000FF0E58EC2AF072EC46F0FF0E58EC2AF006
:108010001200FF0E58EC2AF0B2EC45F0FF0E58ECBF
:108020002AF0C2EC45F0FF0E58EC2AF0B2EC46F014
:10803000FF0E58EC2AF0A2EC45F0FF0E58EC2AF0A7
:108040001200FF0E58EC2AF0A2EC45F0FF0E58EC9F
:108050002AF0A2EC45F0FF0E58EC2AF0F2EC45F0C5
:10806000FF0E58EC2AF01200FF0E58EC2AF092ECAA
:1080700046F0FF0E58EC2AF0C2EC45F0FF0E58EC2B
:108080002AF092EC46F0FF0E58EC2AF092EC46F003
:10809000FF0E58EC2AF01200FF0E58EC2AF082EC8A
:1080A00046F0FF0E58EC2AF0A2EC45F0FF0E58EC1B
:1080B0002AF0F2EC45F0FF0E58EC2AF01200FF0E09
:1080C00058EC2AF0D2EC45F0FF0E58EC2AF0A2EC66
:1080D00045F0FF0E58EC2AF0F2EC45F0FF0E58EC9C
:1080E0002AF012007C0E58EC2AF0820E58EC2AF08E
:1080F000820E58EC2AF0820E58EC2AF07C0E58ECD6
:108100002AF01200000E58EC2AF0840E58EC2AF0E7
:10811000FE0E58EC2AF0800E58EC2AF0000E58ECB7
:108120002AF01200E20E58EC2AF0920E58EC2AF0D7
:10813000920E58EC2AF0920E58EC2AF08C0E58EC65
:108140002AF01200440E58EC2AF0820E58EC2AF065
:10815000920E58EC2AF0920E58EC2AF06C0E58EC65
:108160002AF01200300E58EC2AF0280E58EC2AF0B3
:10817000240E58EC2AF0FE0E58EC2AF0200E58EC93
:108180002AF012004E0E58EC2AF08A0E58EC2AF013
:108190008A0E58EC2AF08A0E58EC2AF0720E58EC2F
:1081A0002AF012007C0E58EC2AF0920E58EC2AF0BD
:1081B000920E58EC2AF0920E58EC2AF0640E58EC0D
:1081C0002AF01200060E58EC2AF0020E58EC2AF0A3
:1081D000C20E58EC2AF0320E58EC2AF00E0E58EC73
:1081E0002AF012006C0E58EC2AF0920E58EC2AF08D
:1081F000920E58EC2AF0920E58EC2AF06C0E58ECC5
:108200002AF012004C0E58EC2AF0920E58EC2AF08C
:10821000920E58EC2AF0920E58EC2AF07C0E58EC94
:108220002AF012003C0E58EC2AF0420E58EC2AF0CC
:10823000420E58EC2AF0420E58EC2AF03C0E58EC54
:108240002AF01200000E58EC2AF0440E58EC2AF0E6
:108250007E0E58EC2AF0400E58EC2AF0000E58EC36
:108260002AF01200720E58EC2AF04A0E58EC2AF04E
:108270004A0E58EC2AF04A0E58EC2AF0440E58ECFC
:108280002AF01200220E58EC2AF04A0E58EC2AF07E
:108290004A0E58EC2AF04A0E58EC2AF0340E58ECEC
:1082A0002AF01200300E58EC2AF0280E58EC2AF072
:1082B000240E58EC2AF07E0E58EC2AF0200E58ECD2
:1082C0002AF012002E0E58EC2AF04A0E58EC2AF032
:1082D0004A0E58EC2AF04A0E58EC2AF0320E58ECAE
:1082E0002AF012003C0E58EC2AF04A0E58EC2AF004
:1082F0004A0E58EC2AF04A0E58EC2AF0300E58EC90
:108300002AF01200060E58EC2AF0020E58EC2AF061
:10831000620E58EC2AF0120E58EC2AF00E0E58ECB1
:108320002AF01200340E58EC2AF04A0E58EC2AF0CB
:108330004A0E58EC2AF04A0E58EC2AF0340E58EC4B
:108340002AF012000C0E58EC2AF0520E58EC2AF0CB
:10835000520E58EC2AF0520E58EC2AF03C0E58EC13
:108360002AF01200C30E58EC2AF0BD0E58EC2AF089
:10837000BD0E58EC2AF0BD0E58EC2AF0C30E58EC96
:108380002AF01200FF0E58EC2AF0BB0E58EC2AF02F
:10839000810E58EC2AF0BF0E58EC2AF0FF0E58EC74
:1083A0002AF012008D0E58EC2AF0B50E58EC2AF087
:1083B000B50E58EC2AF0B50E58EC2AF0BB0E58EC6E
:1083C0002AF01200DD0E58EC2AF0B50E58EC2AF017
:1083D000B50E58EC2AF0B50E58EC2AF0CB0E58EC3E
:1083E0002AF01200CF0E58EC2AF0D70E58EC2AF0E3
:1083F000DB0E58EC2AF0810E58EC2AF0DF0E58EC18
:108400002AF01200D10E58EC2AF0B50E58EC2AF0E2
:10841000B50E58EC2AF0B50E58EC2AF0CD0E58ECFB
:108420002AF01200C30E58EC2AF0B50E58EC2AF0D0
:10843000B50E58EC2AF0B50E58EC2AF0CF0E58ECD9
:108440002AF01200F90E58EC2AF0FD0E58EC2AF032
:108450009D0E58EC2AF0ED0E58EC2AF0F10E58EC77
:108460002AF01200CB0E58EC2AF0B50E58EC2AF088
:10847000B50E58EC2AF0B50E58EC2AF0CB0E58EC9D
:108480002AF01200F30E58EC2AF0AD0E58EC2AF048
:10849000AD0E58EC2AF0AD0E58EC2AF0C30E58EC95
:1084A0002AF01200F80E58EC2AF0240E58EC2AF0AC
:1084B000220E58EC2AF0240E58EC2AF0F80E58EC54
:1084C0002AF01200FE0E58EC2AF0920E58EC2AF018
:1084D000920E58EC2AF0920E58EC2AF06C0E58ECE2
:1084E0002AF012007C0E58EC2AF0820E58EC2AF08A
:1084F000820E58EC2AF0820E58EC2AF0440E58EC0A
:108500002AF01200FE0E58EC2AF0820E58EC2AF0E7
:10851000820E58EC2AF0820E58EC2AF07C0E58ECB1
:108520002AF01200FE0E58EC2AF0920E58EC2AF0B7
:10853000920E58EC2AF0920E58EC2AF0820E58EC6B
:108540002AF01200FE0E58EC2AF0120E58EC2AF017
:10855000120E58EC2AF0120E58EC2AF0020E58ECCB
:108560002AF012007C0E58EC2AF0820E58EC2AF009
:10857000820E58EC2AF0920E58EC2AF0740E58EC49
:108580002AF01200FE0E58EC2AF0100E58EC2AF0D9
:10859000100E58EC2AF0100E58EC2AF0FE0E58EC93
:1085A0002AF01200000E58EC2AF0820E58EC2AF045
:1085B000FE0E58EC2AF0820E58EC2AF0000E58EC11
:1085C0002AF01200600E58EC2AF0800E58EC2AF0C7
:1085D000800E58EC2AF0800E58EC2AF07E0E58ECF3
:1085E0002AF01200FE0E58EC2AF0100E58EC2AF079
:1085F000280E58EC2AF0440E58EC2AF0820E58EC63
:108600002AF01200FE0E58EC2AF0800E58EC2AF0E8
:10861000800E58EC2AF0800E58EC2AF0800E58ECB0
:108620002AF01200FE0E58EC2AF0040E58EC2AF044
:10863000080E58EC2AF0040E58EC2AF0FE0E58EC06
:108640002AF01200FE0E58EC2AF0080E58EC2AF020
:10865000100E58EC2AF0200E58EC2AF0FE0E58ECC2
:108660002AF012007C0E58EC2AF0820E58EC2AF008
:10867000820E58EC2AF0820E58EC2AF07C0E58EC50
:108680002AF01200FE0E58EC2AF0120E58EC2AF0D6
:10869000120E58EC2AF0120E58EC2AF00C0E58EC80
:1086A0002AF012007C0E58EC2AF0820E58EC2AF0C8
:1086B000A20E58EC2AF0420E58EC2AF0BC0E58ECF0
:1086C0002AF01200FE0E58EC2AF0120E58EC2AF096
:1086D000120E58EC2AF0120E58EC2AF0EC0E58EC60
:1086E0002AF012004C0E58EC2AF0920E58EC2AF0A8
:1086F000920E58EC2AF0920E58EC2AF0640E58ECC8
:108700002AF01200020E58EC2AF0020E58EC2AF061
:10871000FE0E58EC2AF0020E58EC2AF0020E58EC2D
:108720002AF012007E0E58EC2AF0800E58EC2AF047
:10873000800E58EC2AF0800E58EC2AF07E0E58EC91
:108740002AF012000E0E58EC2AF0300E58EC2AF0E7
:10875000C00E58EC2AF0300E58EC2AF00E0E58ECF1
:108760002AF012001E0E58EC2AF0E00E58EC2AF007
:10877000180E58EC2AF0E00E58EC2AF01E0E58ECB9
:108780002AF01200C60E58EC2AF0280E58EC2AF0F7
:10879000100E58EC2AF0280E58EC2AF0C60E58ECB1
:1087A0002AF012000E0E58EC2AF0100E58EC2AF0A7
:1087B000E00E58EC2AF0100E58EC2AF00E0E58EC91
:1087C0002AF01200C20E58EC2AF0A20E58EC2AF041
:1087D000920E58EC2AF08A0E58EC2AF0860E58ECCD
:1087E0002AF01200780E58EC2AF0140E58EC2AF0F9
:1087F000120E58EC2AF0140E58EC2AF0780E58ECB1
:108800002AF012007E0E58EC2AF04A0E58EC2AF09C
:108810004A0E58EC2AF04A0E58EC2AF0340E58EC66
:108820002AF012003C0E58EC2AF0420E58EC2AF0C6
:10883000420E58EC2AF0420E58EC2AF0240E58EC66
:108840002AF012007E0E58EC2AF0420E58EC2AF064
:10885000420E58EC2AF0420E58EC2AF03C0E58EC2E
:108860002AF012007E0E58EC2AF04A0E58EC2AF03C
:108870004A0E58EC2AF04A0E58EC2AF0420E58ECF8
:108880002AF012007E0E58EC2AF00A0E58EC2AF05C
:108890000A0E58EC2AF00A0E58EC2AF0020E58EC98
:1088A0002AF012003C0E58EC2AF0420E58EC2AF046
:1088B000420E58EC2AF0520E58EC2AF0340E58ECC6
:1088C0002AF012007E0E58EC2AF0080E58EC2AF01E
:1088D000080E58EC2AF0080E58EC2AF07E0E58ECE0
:1088E0002AF01200000E58EC2AF0420E58EC2AF042
:1088F0007E0E58EC2AF0420E58EC2AF0000E58EC8E
:108900002AF012007E0E58EC2AF0100E58EC2AF0D5
:10891000080E58EC2AF0140E58EC2AF0620E58ECAF
:108920002AF012007E0E58EC2AF0400E58EC2AF085
:10893000400E58EC2AF0400E58EC2AF0400E58EC4D
:108940002AF012007E0E58EC2AF0040E58EC2AF0A1
:10895000080E58EC2AF0040E58EC2AF07E0E58EC63
:108960002AF012007E0E58EC2AF0040E58EC2AF081
:10897000180E58EC2AF0200E58EC2AF07E0E58EC17
:108980002AF012003C0E58EC2AF0420E58EC2AF065
:10899000420E58EC2AF0420E58EC2AF03C0E58ECED
:1089A0002AF012007E0E58EC2AF0120E58EC2AF033
:1089B000120E58EC2AF0120E58EC2AF00C0E58EC5D
:1089C0002AF012003C0E58EC2AF0420E58EC2AF025
:1089D000520E58EC2AF0220E58EC2AF05C0E58EC9D
:1089E0002AF012007E0E58EC2AF0120E58EC2AF0F3
:1089F000120E58EC2AF0120E58EC2AF06C0E58ECBD
:108A00002AF01200440E58EC2AF04A0E58EC2AF0D4
:108A10004A0E58EC2AF04A0E58EC2AF0320E58EC66
:108A20002AF01200020E58EC2AF0020E58EC2AF03E
:108A30007E0E58EC2AF0020E58EC2AF0020E58EC8A
:108A40002AF012003E0E58EC2AF0400E58EC2AF0A4
:108A5000400E58EC2AF0400E58EC2AF03E0E58EC2E
:108A60002AF01200060E58EC2AF0180E58EC2AF0E4
:108A7000600E58EC2AF0180E58EC2AF0060E58EC4E
:108A80002AF012007E0E58EC2AF0200E58EC2AF044
:108A9000100E58EC2AF0200E58EC2AF07E0E58ECFE
:108AA0002AF01200460E58EC2AF0280E58EC2AF054
:108AB000100E58EC2AF0280E58EC2AF0460E58EC0E
:108AC0002AF01200060E58EC2AF0080E58EC2AF094
:108AD000700E58EC2AF0080E58EC2AF0060E58ECEE
:108AE0002AF01200440E58EC2AF0640E58EC2AF0DA
:108AF000540E58EC2AF04C0E58EC2AF0440E58EC68
:108B00002AF01200870E58EC2AF0EB0E58EC2AF0EF
:108B1000ED0E58EC2AF0EB0E58EC2AF0870E58ECCC
:108B20002AF01200810E58EC2AF0B50E58EC2AF00B
:108B3000B50E58EC2AF0B50E58EC2AF0CB0E58ECD6
:108B40002AF01200C30E58EC2AF0BD0E58EC2AF0A1
:108B5000BD0E58EC2AF0BD0E58EC2AF0DB0E58EC96
:108B60002AF01200810E58EC2AF0BD0E58EC2AF0C3
:108B7000BD0E58EC2AF0BD0E58EC2AF0C30E58EC8E
:108B80002AF01200810E58EC2AF0B50E58EC2AF0AB
:108B9000B50E58EC2AF0B50E58EC2AF0BD0E58EC84
:108BA0002AF01200810E58EC2AF0F50E58EC2AF04B
:108BB000F50E58EC2AF0F50E58EC2AF0FD0E58ECA4
:108BC0002AF01200C30E58EC2AF0BD0E58EC2AF021
:108BD000BD0E58EC2AF0AD0E58EC2AF0CB0E58EC36
:108BE0002AF01200810E58EC2AF0F70E58EC2AF009
:108BF000F70E58EC2AF0F70E58EC2AF0810E58ECDC
:108C00002AF01200FF0E58EC2AF0BD0E58EC2AF0A4
:108C1000810E58EC2AF0BD0E58EC2AF0FF0E58ECED
:108C20002AF01200CF0E58EC2AF0BF0E58EC2AF0B2
:108C3000BF0E58EC2AF0BF0E58EC2AF0C10E58ECCB
:108C40002AF01200810E58EC2AF0EF0E58EC2AF0B0
:108C5000F70E58EC2AF0EB0E58EC2AF09D0E58EC6B
:108C60002AF01200810E58EC2AF0BF0E58EC2AF0C0
:108C7000BF0E58EC2AF0BF0E58EC2AF0BF0E58EC8D
:108C80002AF01200810E58EC2AF0FB0E58EC2AF064
:108C9000F70E58EC2AF0FB0E58EC2AF0810E58EC37
:108CA0002AF01200810E58EC2AF0FB0E58EC2AF044
:108CB000E70E58EC2AF0DF0E58EC2AF0810E58EC43
:108CC0002AF01200C30E58EC2AF0BD0E58EC2AF020
:108CD000BD0E58EC2AF0BD0E58EC2AF0C30E58EC2D
:108CE0002AF01200810E58EC2AF0ED0E58EC2AF012
:108CF000ED0E58EC2AF0ED0E58EC2AF0F30E58EC7D
:108D00002AF01200C30E58EC2AF0BD0E58EC2AF0DF
:108D1000AD0E58EC2AF0DD0E58EC2AF0A30E58ECFC
:108D20002AF01200810E58EC2AF0ED0E58EC2AF0D1
:108D3000ED0E58EC2AF0ED0E58EC2AF0930E58EC9C
:108D40002AF01200BB0E58EC2AF0B50E58EC2AF0AF
:108D5000B50E58EC2AF0B50E58EC2AF0CD0E58ECB2
:108D60002AF01200FD0E58EC2AF0FD0E58EC2AF005
:108D7000810E58EC2AF0FD0E58EC2AF0FD0E58EC4E
:108D80002AF01200C10E58EC2AF0BF0E58EC2AF05F
:108D9000BF0E58EC2AF0BF0E58EC2AF0C10E58EC6A
:108DA0002AF01200F90E58EC2AF0E70E58EC2AF0DF
:108DB0009F0E58EC2AF0E70E58EC2AF0F90E58EC0A
:108DC0002AF01200810E58EC2AF0DF0E58EC2AF03F
:108DD000EF0E58EC2AF0DF0E58EC2AF0810E58EC1A
:108DE0002AF01200B90E58EC2AF0D70E58EC2AF0EF
:108DF000EF0E58EC2AF0D70E58EC2AF0B90E58ECCA
:108E00002AF01200F90E58EC2AF0F70E58EC2AF06E
:108E10008F0E58EC2AF0F70E58EC2AF0F90E58ECA9
:108E20002AF01200000E58EC2AF0000E58EC2AF03E
:108E3000040E58EC2AF00A0E58EC2AF0040E58ECF6
:108E40002AF01200000E58EC2AF0000E58EC2AF01E
:108E5000000E58EC2AF0000E58EC2AF0000E58ECE8
:108E60002AF01200FF0E58EC2AF0FF0E58EC2AF000
:108E7000FF0E58EC2AF0FF0E58EC2AF0FF0E58ECCB
:108E80002AF01200280E58EC2AF01200FE0E58ECC0
:108E90002AF0FE0E58EC2AF0000E58EC2AF01200D0
:108EA000000E58EC2AF0000E58EC2AF0000E58EC98
:108EB0002AF01200000EAA6E000EA96E1150A86EC4
:108EC000A69EA69CA684550EA76EAA0EA76EA68285
:108ED000A6B268EF47F0A6941200000EAA6E010E2B
:108EE000A96E1250A86EA69EA69CA684550EA76ECB
:108EF000AA0EA76EA682A6B27BEF47F0A694120038
:108F0000000EAA6E020EA96E1350A86EA69EA69C15
:108F1000A684550EA76EAA0EA76EA682A6B28EEFE5
:108F200047F0A6941200000EAA6E030EA96E14500C
:108F3000A86EA69EA69CA684550EA76EAA0EA76E26
:108F4000A682A6B2A1EF47F0A6941200000EAA6E68
:108F5000040EA96E1550A86EA69EA69CA684550E5A
:108F6000A76EAA0EA76EA682A6B2B4EF47F0A6948B
:108F70001200000EAA6E050EA96E1650A86EA69ECF
:108F8000A69CA684550EA76EAA0EA76EA682A6B2B0
:108F9000C7EF47F0A6941200000EAA6E060EA96E47
:108FA0001750A86EA69EA69CA684550EA76EAA0E64
:108FB000A76EA682A6B2DAEF47F0A6941200000EC2
:108FC000AA6E070EA96E1850A86EA69EA69CA6842F
:108FD000550EA76EAA0EA76EA682A6B2EDEF47F0B9
:108FE000A6941200000EAA6E080EA96E1950A86E63
:108FF000A69EA69CA684550EA76EAA0EA76EA68254
:10900000A6B200EF48F0A6941200000EAA6E090E58
:10901000A96E1A50A86EA69EA69CA684550EA76E91
:10902000AA0EA76EA682A6B213EF48F0A69412006D
:10903000000EAA6E0A0EA96E4C9E4C50A86EA69EFB
:10904000A69CA684550EA76EAA0EA76EA682A6B2EF
:0890500027EF48F0A69412007E
:020000040030CA
:03000100331800B1
:02000500358044
:060008000FC00FE00F40E5
:0200000400F00A
:0C00000008044BBB9B887F7F00000000C1
:00000001FF
